:020000040000FA
:100000004899002045020000690200006B020000D0
:100010006D0200006F020000710200007302000018
:1000200073020000730200007302000073020000FC
:1000300073020000730200002F0300000D4B00004C
:100040003D0D0000470D0000510D00005B0D00004C
:10005000650D00005D10000067100000810F0000BA
:10006000870E0000F50E0000FF0E0000090F0000D3
:10007000130F0000270F0000990C0000A30C0000D4
:10008000AD0C0000B70C0000CB100000BD0F00004D
:10009000C70F0000D10F0000DB0F0000E50F0000CC
:1000A000EF0F00007B0C0000850C00008F0C00009F
:1000B000A90F0000290D00006F0D0000790D000050
:1000C000830D0000711000008B0F0000F90F00007D
:1000D00003100000910E0000F30C0000FD0C000066
:1000E0001F0D00007D0E0000C11000001D0F00005C
:1000F000B7100000AD100000C10C0000CB0C0000D8
:10010000D50C0000DF0C0000150D00008D0D000067
:10011000970D0000A10D0000950F00009F0F00003B
:100120007B100000851000008F1000009910000067
:10013000A31000009B0E0000A50E00000D10000093
:1001400017100000211000002B100000330D0000DC
:10015000590F0000630F0000AF0E0000B90E000041
:10016000AB0D0000B50D00006D0F0000B30F0000D7
:10017000BF0D0000C90D0000D30D0000DD0D000013
:10018000E70D0000F10D0000FB0D0000050E000062
:100190000F0E0000190E0000230E00002D0E0000AF
:1001A000370E0000410E00004B0E0000550E0000FF
:1001B0005F0E0000690E0000770F0000E90C0000E0
:1001C000070D0000EB0E0000351000003F1000008E
:1001D0004910000053100000C30E0000CD0E0000B7
:1001E000310F0000710C00003B0F0000450F0000B4
:1001F0004F0F0000D70E0000E10E0000730E00004C
:10020000DFF80CD000F04CFB00480047058A0000E6
:1002100048990020EFF3108072B67047EFF310801A
:100220007047EFF3108062B6704730BF704780F3BD
:1002300011887047EFF31180704700000138FDD13D
:1002400070470000DFF83000016841F47001016080
:10025000BFF34F8FDFF82400016821F040410160B7
:10026000BFF36F8F06480047FEE7FEE7FEE7FEE7B5
:10027000FEE7FEE7FEE7000088ED00E034EF00E077
:100280000102000072B6704762B67047EFF310804B
:1002900072B6704780F31088704730BF704720BF38
:1002A0007047B0FA80F0704790FAA0F0B0FA80F092
:1002B000704790FAA0F07047EFF3098141B1F1EE79
:1002C000101A40F8041D20ED200A29490A68106020
:1002D0007047B0EC200A02C8E1EE101A25490A68FE
:1002E00010607047EFF3108072B6704780F310888B
:1002F000704721484FF0FF010170002080F309880A
:100300001E48016881F308881D48012101701D48BD
:100310004FF08051016062B6FEE71A484FF08051FD
:100320000160704717484FF080510160704772B606
:10033000EFF3098028B1203880E8F00F0C490968F4
:10034000086000B5104880475DF804EB0F4810497D
:100350000A780270064807490A680260106890E847
:10036000F00F203080F309884EF0F40E62B670472B
:10037000380000204000002022ED00E07000002046
:100380003200002004ED00E0F546000027000020C8
:10039000280000202DE9F05F0546002092469B468C
:1003A00088460646814640241BE02846414647468B
:1003B000224600F02FF853465A46C01A914110D3F6
:1003C00011461846224600F016F82D1A67EB010870
:1003D0004F4622460120002100F00DF817EB0009DE
:1003E0004E41201EA4F10104DFDC484631462A4676
:1003F0004346BDE8F09F202A04DB203A00FA02F1D0
:10040000002070479140C2F1200320FA03F3194302
:1004100090407047202A04DB203A21FA02F00021A4
:10042000704721FA02F3D040C2F120029140084304
:100430001946704740EA01039B0703D009E008C949
:10044000121F08C0042AFAD203E011F8013B00F899
:10045000013B521EF9D27047D2B201E000F8012BE5
:10046000491EFBD270470022F6E710B513460A4634
:1004700004461946FFF7F0FF204610BD30B505468B
:100480002A460B4612F8010B13F8014B08B1A042A3
:10049000F8D01CB1002802D06D1CF1E7284630BD11
:1004A000421C10F8011B0029FBD1801A704700F094
:1004B000004230F000400AD0C10D01F56071C0F378
:1004C000160042EA0151C20840071143704700205C
:1004D0000146704730B5041E71F1000404DB4FF093
:1004E0000044404264EB0101141E73F1000405DB7B
:1004F0001C464FF00043524263EB04038B4208BF9B
:10050000824230BD30B50B46014600202022012436
:1005100009E021FA02F59D4205D303FA02F5491BD1
:1005200004FA02F52844151EA2F10102F1DC30BDE7
:100530002DE9FE4F804681EA0300C00F0C46009073
:1005400021F0004123F00045B8EB0200A94105D29B
:100550004046214690461C460B46024623F000408A
:10056000104347D0270DC7F30A00C3F30A51029086
:10057000401A019040286BDAC3F3130040F4801B4B
:100580000098924620B10023D2EB030A63EB0B0BD9
:1005900001985946C0F140025046FFF72CFF06462D
:1005A0000D4650465946019A00F08CF910EB0800B0
:1005B0006141002487EA115284EAE7731A4340D06C
:1005C000009A62B3019A012A4FEA075215DC001B18
:1005D00061EB02014FF0004202EA0752CDE900420E
:1005E000001C41F5801132462B4600F08CF903B017
:1005F000BDE8F08F40462146F9E7001B61EB0201A0
:10060000001C41F5801300185B412018A2F500176B
:1006100047EB030140EAD570B6196D4111E06D0852
:100620004FEA360645EAC0754FEA0752001B61EBF8
:100630000201001C41F5801149084FEA3000001901
:10064000514132462B4603B0BDE8F04F00F04CB9A3
:100650000098012240000023D0EB020263EBE0731C
:10066000009821464FEAE074B8EB000061EB04010A
:10067000E9E783F000435BE781F0004158E72DE9AB
:10068000FE4F81EA030404F0004421F0004100948D
:100690004FF0000B23F0004350EA01045ED052EA11
:1006A00003045BD0C3F30A54C1F30A552C44A4F2EB
:1006B000F3340194A0FB0254C1F3130141F48011FF
:1006C000C3F3130343F4801301FB024400FB034E06
:1006D000840A970A44EA815447EA8357A4FB0768CF
:1006E00002958D0A05FB07854FEA932C04FB0C54F9
:1006F0002705029D4FEA065847EA1637B5EB08056D
:100700006EEB070C870E920E47EA811742EA8312BE
:10071000A7FB0201B6EB0B0164EB00042B0D43EACF
:100720000C335E1844EB1C50DA465146E7FB0201DD
:10073000C5F313044FEA0B3343EA14534FEA043270
:10074000019C43EA0603A4F10C040294009CCDE949
:1007500000B400F0D8F803B0BDE8F08F00200146E7
:10076000F9E72DE9F04D81EA030404F0004B21F094
:10077000004514464FF0000A23F0004150EA0502FC
:1007800020D054EA01021DD0C5F30A570246C5F332
:100790001303C1F31300C1F30A5640F4801543F468
:1007A0008013A7EB0608101BD64608F2FD3873EB42
:1007B000050002D308F1010801E092185B41B8F18D
:1007C000000F03DA00200146BDE8F08D00204FF451
:1007D0008011064684460EE0171B73EB050705D310
:1007E000121B63EB050306434CEA010C49084FEA70
:1007F000300092185B4150EA0107EDD152EA030044
:1008000012D082EA040083EA0501084305D0101BD8
:10081000AB4106D20122002306E000224FF0004344
:1008200002E06FF0010253101AEB06004CEB085186
:1008300010EB0A0041EB0B01BDE8F04D00F054B89D
:10084000C1F30A52C1F3130140F2FF3341F48011A6
:100850009A4202DA00200146704740F233439A423E
:10086000A2F2334202DC5242FFF7D4BDFFF7C3BD10
:1008700030B5041E71F1000404DB4FF00044404227
:1008800064EB0101141E73F1000405DB1C464FF0FC
:100890000043524263EB0403994208BF904230BDCB
:1008A000064C074D06E0E06840F0010394E80700BD
:1008B00098471034AC42F6D3FFF7A6FC8C9B00009F
:1008C000AC9B0000202A06DBCB17203A41FA02F04D
:1008D00043EAE07306E041FA02F3D040C2F120029D
:1008E000914008431946704710B5141E73F1000477
:1008F00008DA401C41F1000192185B411A4301D112
:1009000020F0010010BD2DE9F04D92469B4611B13B
:10091000B1FA81F202E0B0FA80F220329046FFF79D
:100920006AFD04460F4640EA0A0041EA0B015346BD
:100930005A46084313D0114653EA010019D0C8F1B2
:1009400040025046FFF766FD05460E4650465946A2
:100950004246FFF750FD084305D0012004E0204641
:100960003946BDE8F08D0020054346EAE0762C4389
:1009700037430A986305E40AA0EB08000022FD0A49
:1009800044EA47540A3002D500200146E9E7010550
:1009900010196941DDE9084500196941BDE8F04DCC
:1009A000A2E770B58C1810F8015B15F0070301D1B0
:1009B00010F8013B2A1106D110F8012B03E010F8C2
:1009C000016B01F8016B5B1EF9D12B0705D40023E5
:1009D000521E0DD401F8013BFAE710F8013BCB1A87
:1009E000921C03E013F8015B01F8015B521EF9D57C
:1009F000A142D8D3002070BD0022490801E0521C5A
:100A000049080029FBD10263704701228A40C26075
:100A1000704701228A40C260826801238B401A43DA
:100A20008260704710B50A0C120401F00F04012314
:100A3000A3401A43836A1A43826210BD70B51446FC
:100A4000890045690F268E40B54304F00F068E409D
:100A500035434561056A0F268E40B54303F0030612
:100A60008E403543056204F00F02062A0CD3092A92
:100A70000AD8951FEA00C56930269640B54304F0B0
:100A8000300696403543C56170BD10B503464C0134
:100A900040342344002002E09C6810C2401CDC6803
:100AA00004F480740CB90828F6D310BD0268012341
:100AB0008B401A430260704770B50C4665014035A3
:100AC0002844920005680F269640B54303F00F06B0
:100AD00096403543056085690F269640B543C3F3BC
:100AE000032696403543856146680F25954026EAE2
:100AF0000505C3F30316964035434560C6690F25C7
:100B0000954026EA0505C3F3035696403543C56173
:100B100003F4702575B141690F259540A943C3F3CE
:100B200002459540294341610569012696403543B8
:100B3000056104E0056901269640B543056170BD75
:100B400000B585B0032000214FF400720E4BCDE9B3
:100B50000310CDE90132009003460C4A0C4803F023
:100B6000BFFA032000214FF400720A4BCDE9013295
:100B7000CDE9031005200346074A0090074803F01B
:100B8000AFFA05B000BD0000483900204441002004
:100B9000E16800004841002044490020295B000032
:100BA00000F036F800F0BEFA04464FF47A70B4FB59
:100BB000F0F5284603F0BEFF00F06EFB03F064FA88
:100BC00002F054FF01F0F6FD05F03EFB05F012FFC8
:100BD000FFF7B6FF13E0012001F00AFA002001F050
:100BE00019FA4FF47A7003F089FD002001F000FA41
:100BF000012001F00FFA4FF47A7003F07FFDEAE76D
:100C0000704770477047704770477047704770472C
:100C100010B500F05FFA00F0DFFA10BD10B5044621
:100C2000702C04D204F11001C8B200F03BFB10BDDF
:100C300070B50446002600BF00BFFFF727FB06463D
:100C400000BF00BF03F07CF800BF00BF3046FFF7D5
:100C500021FB00BF00BF702C04D2044850F8245080
:100C600005B1A84703F086F870BD000050060020CB
:100C700010B56920FFF7DCFF10BD10B51920FFF794
:100C8000D7FF10BD10B51A20FFF7D2FF10BD10B569
:100C90001B20FFF7CDFF10BD10B50E20FFF7C8FFDA
:100CA00010BD10B50F20FFF7C3FF10BD10B5102009
:100CB000FFF7BEFF10BD10B51120FFF7B9FF10BD43
:100CC00010B52E20FFF7B4FF10BD10B52F20FFF791
:100CD000AFFF10BD10B53020FFF7AAFF10BD10B553
:100CE0003120FFF7A5FF10BD10B55F20FFF7A0FF73
:100CF00010BD10B52620FFF79BFF10BD10B52720B3
:100D0000FFF796FF10BD10B56020FFF791FF10BDF3
:100D100000BFFEE710B53220FFF78AFF10BD10B507
:100D20002820FFF785FF10BD10B51D20FFF780FFBD
:100D300010BD10B54320FFF77BFF10BD10B500209C
:100D4000FFF776FF10BD10B50120FFF771FF10BD52
:100D500010B50220FFF76CFF10BD10B50320FFF7A0
:100D600067FF10BD10B50420FFF762FF10BD10B57E
:100D70001E20FFF75DFF10BD10B51F20FFF758FFC5
:100D800010BD10B52020FFF753FF10BD10B5332064
:100D9000FFF74EFF10BD10B53420FFF749FF10BD1F
:100DA00010B53520FFF744FF10BD10B54820FFF700
:100DB0003FFF10BD10B54920FFF73AFF10BD10B539
:100DC0004C20FFF735FF10BD10B54D20FFF730FF69
:100DD00010BD10B54E20FFF72BFF10BD10B54F20F2
:100DE000FFF726FF10BD10B55020FFF721FF10BD03
:100DF00010B55120FFF71CFF10BD10B55220FFF7B2
:100E000017FF10BD10B55320FFF712FF10BD10B52E
:100E10005420FFF70DFF10BD10B55520FFF708FF58
:100E200010BD10B55620FFF703FF10BD10B55720B9
:100E3000FFF7FEFE10BD10B55820FFF7F9FE10BDFC
:100E400010B55920FFF7F4FE10BD10B55A20FFF77A
:100E5000EFFE10BD10B55B20FFF7EAFE10BD10B528
:100E60005C20FFF7E5FE10BD10B55D20FFF7E0FE4A
:100E700010BD10B56F20FFF7DBFE10BD10B52920A7
:100E8000FFF7D6FE10BD10B50820FFF7D1FE10BD4C
:100E900010B52520FFF7CCFE10BD10B53D20FFF7A3
:100EA000C7FE10BD10B53E20FFF7C2FE10BD10B545
:100EB0004620FFF7BDFE10BD10B54720FFF7B8FE76
:100EC00010BD10B56620FFF7B3FE10BD10B567204A
:100ED000FFF7AEFE10BD10B56D20FFF7A9FE10BDE7
:100EE00010B56E20FFF7A4FE10BD10B56120FFF70E
:100EF0009FFE10BD10B50920FFF79AFE10BD10B57A
:100F00000A20FFF795FE10BD10B50B20FFF790FEED
:100F100010BD10B50C20FFF78BFE10BD10B52B20B7
:100F2000FFF786FE10BD10B50D20FFF781FE10BD46
:100F300010B56820FFF77CFE10BD10B56A20FFF7E2
:100F400077FE10BD10B56B20FFF772FE10BD10B517
:100F50006C20FFF76DFE10BD10B54420FFF768FE52
:100F600010BD10B54520FFF763FE10BD10B54A2037
:100F7000FFF75EFE10BD10B55E20FFF759FE10BDF5
:100F800010B50720FFF754FE10BD10B52220FFF763
:100F90004FFE10BD10B53620FFF74AFE10BD10B54C
:100FA0003720FFF745FE10BD10B51C20FFF740FEAF
:100FB00010BD10B54B20FFF73BFE10BD10B5132040
:100FC000FFF736FE10BD10B51420FFF731FE10BD3F
:100FD00010B51520FFF72CFE10BD10B51620FFF739
:100FE00027FE10BD10B51720FFF722FE10BD10B56B
:100FF0001820FFF71DFE10BD10B52320FFF718FEC7
:1010000010BD10B52420FFF713FE10BD10B53F2012
:10101000FFF70EFE10BD10B54020FFF709FE10BD12
:1010200010B54120FFF704FE10BD10B54220FFF7B8
:10103000FFFD10BD10B56220FFF7FAFD10BD10B521
:101040006320FFF7F5FD10BD10B56420FFF7F0FD3C
:1010500010BD10B56520FFF7EBFD10BD10B50520E4
:10106000FFF7E6FD10BD10B50620FFF7E1FD10BD4E
:1010700010B52120FFF7DCFD10BD10B53820FFF7BB
:10108000D7FD10BD10B53920FFF7D2FD10BD10B54A
:101090003A20FFF7CDFD10BD10B53B20FFF7C8FD8E
:1010A00010BD10B53C20FFF7C3FD10BD10B52D20BD
:1010B000FFF7BEFD10BD10B52C20FFF7B9FD10BD28
:1010C00010B52A20FFF7B4FD10BD10B51220FFF7B0
:1010D000AFFD10BD10B5002404E0E0B2034900F0FC
:1010E00007F8641C702CF8D310BD0000110D00002F
:1010F00070B504460D460026702C10D200BF00BF0C
:10110000FFF7C4F8064600BF00BF054840F824506A
:1011100000BF00BF3046FFF7BDF800BF00BF70BD85
:10112000500600202DE9F043DFF89CC0DCF8B0C089
:10113000CCF3007CBCF1000F3ED0DFF88CC0DCF8B3
:1011400060C1CCF38A26DFF880C0DCF860C1CCF344
:101150000A0303EB9622DFF870C0DCF864C1CCF31D
:101160000424DFF864C0DCF864C10CF01F05DFF86C
:1011700058C0DCF8B0C0CCF3036111B1032904D12D
:1011800001E0124902E0124900E000BF00BF01FB8C
:1011900002F804F1010C05F101090CFB09FCB8FB94
:1011A000FCF0DFF824C0DCF8B0C0CCF3090C0CF183
:1011B0000107B0FBF7F000E00020DFF818C0CCF822
:1011C0000000BDE8F083000000E00F400024F400C0
:1011D00040787D01080000202948C06F20F01C00E5
:1011E0002749C8670846C06F40F01000C867244808
:1011F000C0300068234908402149C1F8C000204898
:10120000C0300068204908431D49C03108604806C5
:101210001B49B03108604FF04C70086060201B49DA
:10122000086004201649C1F864011848A038006815
:10123000144908401249C1F8C0001448A038006899
:10124000134908430E49C1F8C0000846D0F86001B0
:1012500040F40000C1F8600100BF0C48083000688D
:1012600000F0010080F001000028F6D10448B03001
:101270000068084908430249C1F8B00070470000FF
:1012800000E00F4010FC10FC8100010060E10F4005
:10129000850185010300009010B500F0F9F800F019
:1012A000BFF810BD2DE9F04104464FF00008102CA6
:1012B0006BD2DFE804F0080E0F1014293E090A0B68
:1012C0000C11120D135300BF00BF00BF00BF00BFC1
:1012D00089E000BF00BF00BF00BF00BF83E000BFC8
:1012E00000BFFEF7D3FF804600BF00BF3F48006845
:1012F00040F480303D49086000BF00BF4046FEF723
:10130000C9FF00BF00BF6EE000BF00BFFEF7BEFF19
:10131000804600BF00BF3548006840F400303349C4
:10132000086000BF00BF4046FEF7B4FF00BF00BF2B
:1013300059E000BF00BFFEF7A9FF804600BF00BF15
:101340002A48006840F480202849086000BF00BF98
:101350004046FEF79FFF00BF00BF44E000BF00BF54
:10136000FEF794FF804600BF00BF4FF0E020006909
:1013700040F001004FF0E021086100BF00BF40468F
:10138000FEF788FF00BF00BF2DE04FF0E02040686F
:10139000401C102101EB4010C7B2BC4222DAA4F17C
:1013A0001000C11700EBD161C1F34715C11700EB65
:1013B000D1614911A0EB4111CEB200BF00BFFEF7D1
:1013C00065FF804600BF00BF0120B040A90001F1C9
:1013D000E021C1F8000100BF00BF4046FEF75AFF00
:1013E00000BF00BF00BF00BFBDE8F08124ED00E0FA
:1013F00010B5002400BF00BFFEF748FF044600BF41
:1014000000BF1021054802F027FB00BF00BF2046A7
:10141000FEF740FF00BF00BF10BD0000F801002034
:1014200010B5FFF7E5FF10BD2DE9F04105460C466C
:10143000002714B900BF00F029F81DB90A20208048
:10144000BDE8F0811021284604F0E1FA0646102E8E
:1014500015D200BF00BFFEF719FF074600BF00BF4F
:1014600010222946084804F0AFFA00BF00BF3846F2
:10147000FEF710FF00BF00BF0020208002E04FF405
:101480007A70208000BFDBE7F801002000BFFEE794
:1014900010B500200249086000F00AF810BD0000F5
:1014A0000000002001490860704700000000002093
:1014B00010B50A48006840F08070084908600020B4
:1014C000074948600846006840F001000860FFF7DF
:1014D00029FE04462046FFF7E5FF10BDFCED00E0C5
:1014E000001000E010B50220FEF7A8FE05F03EFB5C
:1014F0000B48C46904F00C0008B1022010BD094873
:1015000004F0CAFA0220FEF799FE05F02FFB04480A
:10151000C46904F00C0008B10220EFE70020EDE7F9
:1015200000F00A40005800F00148006870470000D1
:10153000A001002002F001031BB1D0F800340B43DE
:1015400002E0D0F800348B43C0F8003402F002030C
:101550001BB1D0F820340B4302E0D0F820348B4389
:10156000C0F8203470470000F0B55F4D2D685F4E25
:1015700035405F4EB5421AD0002416E00125A54043
:101580000D4085B1D0F8C45F67000326BE40B54367
:10159000C0F8C45FD0F8C45F6700C2F34116BE4014
:1015A0003543C0F8C45F651CECB2082CE6DB02F0E2
:1015B00001051DB1D0F800550D4302E0D0F80055EB
:1015C0008D43C0F8005502F002051DB1D0F8045556
:1015D0000D4302E0D0F804558D43C0F8045502F0E5
:1015E00004051DB1D0F808550D4302E0D0F80855A8
:1015F0008D43C0F8085502F008051DB1D0F8185504
:101600000D4302E0D0F818558D43C0F81855364DFB
:101610002D68364E3540364EB5420BD002F01005DF
:101620001DB1D0F83C550D4302E0D0F83C558D4338
:10163000C0F83C5503F001051DB1D0F80C550D4321
:1016400002E0D0F80C558D43C0F80C5503F00205AC
:101650001DB1D0F810550D4302E0D0F810558D4360
:10166000C0F8105503F004051DB1D0F814550D4312
:1016700002E0D0F814558D43C0F8145503F0080566
:101680001DB1D0F81C550D4302E0D0F81C558D4318
:10169000C0F81C55144D2D68144E3540144EB542FB
:1016A00017D003F400751DB1D0F844550D4302E086
:1016B000D0F844558D43C0F8445503F440751DB12E
:1016C000D0F840550D4302E0D0F840558D43C0F8A6
:1016D00040551BB9D0F828550D4302E0D0F82855E5
:1016E0008D43C0F82855F0BD00E00F400000FF70AA
:1016F0000000051010B50146C1F307400F4BDB6E2B
:1017000001248440234033B1012303EB40030C4CFC
:1017100054F8230003E04300094C54F82300C1F3BC
:101720000722D0F82C350F249440A34301F00F0476
:1017300094402343C0F82C3510BD000000E00F405A
:10174000C09300000246002000EB81001058704753
:1017500030B504460D46002229462046FFF7EAFE32
:101760000023012229462046FFF7FEFE30BD30B59A
:1017700004460D46022229462046FFF7DBFE0823D9
:10178000012229462046FFF7EFFE30BD30B5044662
:101790000D46022229462046FFF7CCFE08230122EF
:1017A00029462046FFF7E0FE30BD002303EB81030E
:1017B000C250704770B50546284600F0E9F844B2BB
:1017C000002C02DA4FF0FF3070BD284600F086F89A
:1017D00044B2002C02DA4FF0FF30F5E7284600F063
:1017E00050F844B2002C02DA4FF0FF30ECE7284604
:1017F00000F01AF844B2002C02DA4FF0FF30E3E7B1
:10180000284600F098F844B2002C02DA4FF0FF307E
:10181000DAE7284600F0E8F844B2002C02DA4FF08C
:10182000FF30D1E70020CFE77CB5044603200190CC
:1018300000200090A07D012301AA6F21E669B04736
:1018400045B2002D02DA4FF0FF307CBDA07D0123B0
:101850006A466F21A669B04745B2002D02DA4FF003
:10186000FF30F2E79DF8000000F00F009DF8001037
:10187000C1F3011101EB810100EB4101A1710020D5
:10188000E3E77CB504460220019000200090A07D93
:10189000012301AA6F21E669B04745B2002D02DAA3
:1018A0004FF0FF307CBDA07D01236A466F21A66901
:1018B000B04745B2002D02DA4FF0FF30F2E79DF855
:1018C000000000F00F009DF80010C1F3011101EBC2
:1018D000810100EB410161710020E3E77CB5044622
:1018E0000120019000200090A07D012301AA6F211A
:1018F000E669B04745B2002D02DA4FF0FF307CBDFB
:10190000A07D01236A466F21A669B04745B2002D2C
:1019100002DA4FF0FF30F2E79DF8000000F00F0010
:101920009DF80010C1F3021101EB810100EB4101B0
:1019300021710020E3E77CB50446042001900020DB
:101940000090A07D012301AA6F21E669B04745B24E
:10195000002D02DA4FF0FF307CBDA07D01236A46E6
:101960006F21A669B04745B2002D02DA4FF0FF3073
:10197000F2E79DF8000000F00F009DF80010C1F3A1
:10198000001101EB810100EB4101E1710020E3E76F
:101990007CB50446002001900090A07D012301AA9F
:1019A0006F21E669B04745B2002D02DA4FF0FF30F3
:1019B0007CBDA07D01236A466F21A669B04745B270
:1019C000002D02DA4FF0FF30F2E79DF8000000F042
:1019D0000F009DF80010C1F3021101EB810100EB33
:1019E0004101E1700020E3E77CB504460520019049
:1019F00000200090A07D012301AA6F21E669B04775
:101A000045B2002D02DA4FF0FF307CBDA07D0123EE
:101A10006A466F21A669B04745B2002D02DA4FF041
:101A2000FF30F2E79DF8000000F00F009DF8001075
:101A3000090901EB810100EB41000549098801EB2F
:101A4000C10202EB011100EB810020810020DCE7E4
:101A50007E010020042806D11949096841F480312B
:101A6000174A11602BE0052806D11549096841F491
:101A70000031134A116022E0062806D11049096896
:101A800041F480210E4A116019E00F2808D14FF06F
:101A9000E021096941F002014FF0E02211610EE0FE
:101AA00010280CD3A0F1100101F01F020121914078
:101AB000A0F110025209034B53F822201160704725
:101AC00024ED00E00C95000010B5FEF7AAFB08B16C
:101AD000012010BD0020FCE710B50A4683080A4C1F
:101AE00054F8233019688307DC0EFF23A340994381
:101AF0008307DB0E02FA03F319438308024C54F800
:101B00002330196010BD00007094000010B500244F
:101B100002F016F9FEF7E6FB044600210948FEF73D
:101B200074FF094A00210748FEF7AFFF002007496C
:101B300008700120064908702046FEF7D7FB02F026
:101B400019F910BD00800340C0220020760000205B
:101B50007700002010B5002402F0F2F8FEF7C2FB77
:101B6000044601210948FEF750FF094A01210748B0
:101B7000FEF78BFF00200749087001200649087016
:101B80002046FEF7B3FB02F0F5F810BD00800340DD
:101B9000E0220020780000207900002010B5002409
:101BA00002F0CEF8FEF79EFB044600210948FEF73E
:101BB0002CFF094A00210748FEF767FF002007496C
:101BC00008700120064908702046FEF78FFB02F0DE
:101BD000D1F810BD00900340002300207A000020BF
:101BE0007B00002070B504460D4615B94FF0FF305C
:101BF00070BD3748005D082855D2DFE800F0041DAD
:101C000036373851525300BF324800780028FBD194
:101C100001203049087000202F49087000212F480A
:101C2000FEF7F3FE00212D48FEF7FCFE00BF2A4818
:101C300000780028FBD036E000BF29480078002853
:101C4000FBD1012026490870002026490870012197
:101C50002248FEF7DAFE01212048FEF7E3FE00BF2E
:101C6000204800780028FBD01DE01CE01BE000BFEE
:101C70001D4800780028FBD101201B490870002076
:101C80001A49087000211A48FEF7BFFE00211848C3
:101C9000FEF7C8FE00BF154800780028FBD002E020
:101CA00001E000E000BF00BF124850F8240000EE41
:101CB000100AB8EE400ADFED100A20EE200ADFED30
:101CC0000F0A80EE201A85ED001A002090E7000030
:101CD0007C00002076000020770000200080034078
:101CE00078000020790000207A0000207B0000208E
:101CF00000900340C022002000404E450000804577
:101D000010B5A4480078012801D1002010BDA248D8
:101D100003F08CFEA048401C03F088FE9F4803F0AF
:101D200085FE08219E48FFF713FD9C4803F07EFEC8
:101D300004219B48FFF70CFD984803F077FE022131
:101D40009748FFF705FD954803F070FE0121944880
:101D5000FFF7FEFC9148401E03F068FE8021914889
:101D6000FFF7F6FC8D48401E03F060FE40218D48D1
:101D7000FFF7EEFC8948401E03F058FE20218948F9
:101D8000FFF7E6FC8548401E03F050FE1021854811
:101D9000FFF7DEFC814803F049FE20218048FFF771
:101DA000D7FC7E4803F042FE10217D48FFF7D0FCAF
:101DB0007A48C01E03F03AFE10217B48FFF7C8FCAA
:101DC0007648C01E03F032FE20217748FFF7C0FCA2
:101DD0007248401D03F02AFE01217448FFF7B8FC49
:101DE0006E48401D03F022FE02217048FFF7B0FC50
:101DF0006A48401D03F01AFE04216C48FFF7A8FC56
:101E00006648401D03F012FE08216848FFF7A0FC59
:101E100000231A4619466648FEF710FE01230022E9
:101E200019466348FEF70AFE00231A461946614820
:101E3000FEF704FE08215E48FEF7DEFD08215D483E
:101E4000FEF7DAFD00231A4619465948FEF734FE1C
:101E500001231A4600215648FEF72EFE02231A4699
:101E600000215348FEF728FE03231A46002150485C
:101E7000FEF722FE04231A4600214D48FEF71CFE01
:101E800005231A4600214A48FEF716FE06231A4685
:101E900000214748FEF710FE67230722002144482F
:101EA000FEF70AFE0823002201214148FEF704FE46
:101EB0000923012211463E48FEF7FEFD0A230222B5
:101EC00001213B48FEF7F8FD6B230322012138482E
:101ED000FEF7F2FD4FF48073002211463548FEF7FD
:101EE000EBFD40F20113012200213248FEF7E4FD30
:101EF0004FF48173022200212E48FEF7DDFD40F2EF
:101F00006313032200212B48FEF7D6FD2A490E2039
:101F1000FFF7EEF829490F20FFF7EAF828492E20AD
:101F2000FFF7E6F80E20FEF779FE0F20FEF776FEAB
:101F30002E20FEF773FE00211D48FEF76AFD0121E9
:101F40001B48FEF766FD00211A48FEF762FD1E20C1
:101F5000FFF780FD1F20FFF77DFD3E20FFF77AFD94
:101F600000211348FEF7A2FD01211148FEF79EFD56
:101F700000211048FEF79AFD00210D48FEF745FDAF
:101F800001210B48FEF741FD00210A48FEF73DFD07
:101F90000020BBE690000020003800F0040800F0AC
:101FA0000040024000700040005000400010064019
:101FB00000800340009003400D1B0000551B0000F3
:101FC0009D1B000010B5084803F030FD00BF064817
:101FD00003F046FD0028FAD0FFF784FA04460CB15E
:101FE00000BFFEE710BD0000005800F07047000081
:101FF00010B504462CB9012211460548FFF7D5FB60
:1020000004E0FE2201210248FFF7CFFB10BD0000D3
:102010000070004010B504462CB902221146054854
:10202000FFF7C3FB04E0FD2202210248FFF7BDFBDE
:1020300010BD00000070004010B50E4803F0F6FC23
:10204000012211460C48FFF775FA082301221146B8
:102050000948FFF789FA074803F0E8FC012202214A
:102060000548FFF767FA0823012202210248FFF71B
:102070007BFA10BD030800F00070004070B5044604
:102080000D46042C02DB4FF0FF3070BD04EB440022
:10209000224911F8200010B94FF0FF30F5E774B96C
:1020A00035B9F72208214FF04020FFF77EFB32E0E0
:1020B000082211464FF04020FFF777FB2BE0012C60
:1020C0000CD12DB9EF2210211548FFF76EFB22E04D
:1020D000102211461248FFF768FB1CE0022C0CD1BD
:1020E0002DB9FB2204210F48FFF75FFB13E0042208
:1020F00011460C48FFF759FB0DE0032C0BD12DB90D
:10210000FB2204210848FFF750FB04E0042211469B
:102110000548FFF74AFB0020B7E700001023002026
:102120000050004000700040005002402DE9FE4386
:1021300004460F4690461E460A9D042C03DA042DE1
:1021400001DB102D03DD4FF0FF30BDE8FE8300BF43
:1021500004EB4400A54901EB8000C07A0128F7D0C8
:10216000002004EB4401A14A02F82100002C48D1D0
:102170009F4803F05BFC9F4803F058FC9D4803F028
:1021800055FC9C4803F052FC9A4803F04FFC40F683
:102190000F00FFF7AFFA40F60F40FFF7ABFA41F23E
:1021A0000F00FFF7A7FA41F20F40FFF7A3FA04214F
:1021B0004FF04020FFF7DBFA08214FF04020FFF7F7
:1021C000D6FA10214FF04020FFF7D1FA20214FF02E
:1021D0004020FFF7CCFA03F0A1FC814643463A4683
:1021E00049468548CDE9006503F09DFB824803F030
:1021F000E6FB00BF02A9804803F0C9FB0028F9D123
:10220000D6E0012C45D17A48401C03F00FFC7948F8
:10221000401C03F00BFC7748401C03F007FC75489A
:10222000001D03F003FC7348001D03F0FFFB73481F
:10223000FFF760FA7248FFF75DFA7248FFF75AFA43
:102240007148FFF757FA20217048FFF790FA1021E4
:102250006E48FFF78CFA10216D48FFF788FA2021AD
:102260006B48FFF784FA03F059FC814643463A462F
:1022700049466848CDE9006503F055FB654803F021
:102280009EFB00BF02A9634803F081FB0028F9D13F
:102290008EE0022C45D15648801C03F0C7FB554800
:1022A000C01C03F0C3FB5348C01C03F0BFFB5148E4
:1022B000C01C03F0BBFB4F48C01C03F0B7FB5648E3
:1022C000FFF718FA5548FFF715FA5548FFF712FAC5
:1022D0005448FFF70FFA08215348FFF748FA042142
:1022E0005148FFF744FA02214F48FFF740FA012115
:1022F0004D48FFF73CFA03F011FC814643463A464D
:1023000049464A48CDE9006503F00DFB474803F014
:1023100056FB00BF02A9454803F039FB0028F9D15C
:1023200046E0032C44D13248C01C03F07FFB314807
:10233000401D03F07BFB2F48401D03F077FB2D4829
:10234000401D03F073FB2B48401D03F06FFB384822
:10235000FFF7D0F93748FFF7CDF93748FFF7CAF94B
:102360003648FFF7C7F908213548FFF700FA04217E
:102370003348FFF7FCF902213148FFF7F8F9012152
:102380002F48FFF7F4F903F0C9FB814643463A466C
:1023900049462C48CDE9006503F0C5FA294803F009
:1023A0000EFB00BF02A9274803F0F1FA0028F9D17B
:1023B00004EB44000D4901EB800080F8098004EB38
:1023C000440001EB8000857204EB440001EB8000C7
:1023D000466004EB440001EB80000772012004EB2F
:1023E0004401024A02F821000020AEE6102300203A
:1023F000001C00F0000800F0008000400F140100F5
:102400000F1001000F1004000F14040000500040D2
:1024100000400240009000400F0C03000F08030032
:102420000F0403000F0003000070004000A00040F4
:102430000E0C05000E0805000E0405000E00050038
:102440000050024000B000402DE9FC4704460E4613
:10245000174698460A9D042C03DB4FF0FF30BDE879
:10246000FC8745B12878042802DB2878102802DD93
:102470004FF0FF30F3E704EB44007D4911F82000F2
:1024800010B94FF0FF30EAE700BF04EB4400784991
:1024900001EB8000C07A0128F7D0002004EB440152
:1024A000734A02F821002EB1307804EB440102EBAC
:1024B0008101087237B1387804EB44016C4A02EBB1
:1024C00081014872B8F1000F07D004EB4401684A5B
:1024D00002EB8101D8F80000486035B1287804EBA0
:1024E0004401634A02EB8101887264BB00BF61480A
:1024F00003F014FA0028FAD15E4803F05BFA03F007
:102500000DFB814604EB4400594901EB8000807AC1
:1025100004EB4401564A02EB81014968CDE9001001
:1025200004EB4400114601EB8000437A04EB4400C5
:1025300001EB8000027A49464E4803F0F4F94D4819
:1025400003F03DFA8BE0012C2CD100BF4A4803F088
:10255000E5F90028FAD1484803F02CFA03F0DEFA36
:10256000814604EB4400424901EB8000807A04EB91
:1025700044013F4A02EB81014968CDE9001004EBB8
:102580004400114601EB8000437A04EB440001EB68
:102590008000027A4946384803F0C5F9364803F00E
:1025A0000EFA5CE0022C2CD100BF344803F0B6F9DF
:1025B0000028FAD1314803F0FDF903F0AFFA814663
:1025C00004EB44002A4901EB8000807A04EB4401CB
:1025D000274A02EB81014968CDE9001004EB440071
:1025E000114601EB8000437A04EB440001EB8000CC
:1025F000027A4946214803F096F9204803F0DFF9B2
:102600002DE0032C2BD100BF1D4803F087F90028D3
:10261000FAD11B4803F0CEF903F080FA814604EBAF
:102620004400134901EB8000807A04EB4401104A16
:1026300002EB81014968CDE9001004EB440011462A
:1026400001EB8000437A04EB440001EB8000027A46
:1026500049460B4803F067F9094803F0B0F9012037
:1026600004EB4401024A02F821000020F7E60000D2
:1026700010230020008000400090004000A0004097
:1026800000B00040F8B504460E4615460020009004
:102690000027042C00DA15B94FF0FF30F8BD04EB29
:1026A00044003F4911F82000012802D04FF0FF30CC
:1026B000F4E7012004EB4401394A02EB8101C872BE
:1026C000FDF710FE0746ACB900BF6946354803F078
:1026D0005EF90028F9D13146324803F063F900BFB2
:1026E000304803F01BF90028FAD169462D4803F061
:1026F00045F946E0012C15D100BF69462A4803F090
:1027000046F90028F9D13146274803F04BF900BFBC
:10271000254803F003F90028FAD16946224803F05E
:102720002DF92EE0022C15D100BF69461F4803F099
:102730002EF90028F9D131461C4803F033F900BFC7
:102740001A4803F0EBF80028FAD16946174803F05D
:1027500015F916E0032C14D100BF6946144803F0A4
:1027600016F90028F9D13146114803F01BF900BFD2
:102770000F4803F0D3F80028FAD169460C4803F05B
:10278000FDF8009828703846FDF7B0FD002004EBF6
:102790004401034A02EB8101C87200BF7EE70000DA
:1027A00010230020008000400090004000A0004066
:1027B00000B0004010B5FFF719FCFFF73DFCFFF734
:1027C00083F9FFF7FFFB10BD70B5002401F0B8FAE4
:1027D000FDF788FD04460121124804F0A8F90546DA
:1027E0002946104804F09DF910E00E4804F041F924
:1027F0000D4908700D48407D012807D10C4800683C
:1028000020B1084600780A4909688847054804F05D
:1028100042F90028E9D12046FDF768FD01F0AAFA47
:1028200070BD000000C0004094000020BC000020EB
:102830009C00002070B5002401F082FAFDF752FDE3
:1028400004460121124804F072F905462946104851
:1028500004F067F911E00E4804F00BF90D49087017
:102860000D4890F82D00012807D10C48006820B1D0
:1028700008460078094909688847054804F00BF9BB
:102880000028E8D12046FDF731FD01F073FA70BD54
:1028900000D0004095000020BC000020A0000020D7
:1028A00070B5002401F04CFAFDF71CFD044601212F
:1028B000124804F03CF905462946104804F031F965
:1028C00011E00E4804F0D5F80D4908700D4890F855
:1028D0004500012807D10C48006820B1084600785F
:1028E000094909688847054804F0D5F80028E8D167
:1028F0002046FDF7FBFC01F03DFA70BD00E0004012
:1029000096000020BC000020A400002070B5002428
:1029100001F016FAFDF7E6FC04460121124804F026
:1029200006F905462946104804F0FBF811E00E4868
:1029300004F09FF80D4908700D4890F85D000128DB
:1029400007D10C48006820B1084600780949096899
:102950008847054804F09FF80028E8D12046FDF795
:10296000C5FC01F007FA70BD00F0004097000020A0
:10297000BC000020A800002070B5002401F0E0F9A0
:10298000FDF7B0FC04460121124804F0D0F80546DA
:102990002946104804F0C5F811E00E4804F069F823
:1029A0000D4908700D4890F87500012807D10C48B2
:1029B000006820B108460078094909688847054839
:1029C00004F069F80028E8D12046FDF78FFC01F0FB
:1029D000D1F970BD0000014098000020BC0000202B
:1029E000AC00002070B5002401F0AAF9FDF77AFCD4
:1029F00004460121124804F09AF805462946104879
:102A000004F08FF811E00E4804F033F80D49087017
:102A10000D4890F88D00012807D10C48006820B1BE
:102A200008460078094909688847054804F033F8E2
:102A30000028E8D12046FDF759FC01F09BF970BD54
:102A40000010014099000020BC000020B0000020D0
:102A500070B5002401F074F9FDF744FC044601212F
:102A6000124804F064F805462946104804F059F865
:102A700011E00E4803F0FDFF0D4908700D4890F875
:102A8000A500012807D10C48006820B1084600784D
:102A9000094909688847054803F0FDFF0028E8D187
:102AA0002046FDF723FC01F065F970BD00200140D0
:102AB0009A000020BC000020B400002070B5002463
:102AC00001F03EF9FDF70EFC04460121124804F026
:102AD0002EF805462946104804F023F811E00E4868
:102AE00003F0C7FF0D4908700D4890F8BD0001289C
:102AF00007D10C48006820B10846007809490968E8
:102B00008847054803F0C7FF0028E8D12046FDF7B5
:102B1000EDFB01F02FF970BD003001409B0000205B
:102B2000BC000020B80000202DE9F04704460D4607
:102B300016461F46DDF82080082C03DB4FF0FF30DF
:102B4000BDE8F087B5F5965F18D0B5F5165F15D0DE
:102B5000B5F5615F12D0B5F5964F0FD0B5F5164FAC
:102B60000CD04DF6C020854208D0B5F5614F05D098
:102B7000B5F5E13F02D04FF0FF30E1E704EB440050
:102B8000FE4901EBC0004560052E06D0062E0CD094
:102B9000072E12D0082E20D117E0002004EB4401AC
:102BA000F64A02EBC10188601AE0202004EB4401E0
:102BB000F24A02EBC101886012E0402004EB4401BC
:102BC000EE4A02EBC10188600AE0602004EB440198
:102BD000EA4A02EBC101886002E04FF0FF30AFE744
:102BE00000BF012F02D0022F10D107E0002004EB1C
:102BF0004401E24A02EBC101C8600AE0082004EB8C
:102C00004401DE4A02EBC101C86002E04FF0FF3030
:102C100096E700BFB8F1000F06D0B8F1010F0BD056
:102C2000B8F1020F18D10FE0002004EB4401D34AA1
:102C300002EBC101086112E0062004EB4401CF4A17
:102C400002EBC10108610AE0022004EB4401CB4A17
:102C500002EBC101086102E04FF0FF3070E700BFF6
:102C600000BF04EB4400C54901EBC000007D012812
:102C7000F7D004EB440001EBC000407D0128F0D008
:102C8000002004EB4401BD4A02F83100002C7DD144
:102C9000BB4802F0CBFEBB4802F0C8FEB94802F0C8
:102CA000C5FE0120FEF726FD40F20140FEF722FDA1
:102CB00001214FF04020FEF769FD02214FF0402036
:102CC000FEF764FD02F02AFF824604EB4400AB49A4
:102CD00001EBC000806804EB4401DFF8A0C20CEBFC
:102CE000C101C968084304EB44010CEBC101096947
:102CF00040EA010304EB4400614601EBC000514689
:102D00004268A14803F0CDFE04EB44009B4901EB6F
:102D1000C0004078022816D19A4802F087FE0122AE
:102D200002214FF04020FEF705FC4FF4847301228E
:102D300002214FF04020FEF717FCFD2202214FF048
:102D40004020FEF732FD91490520FEF7D1F905201C
:102D5000FDF764FF1520FEF77DFE60211520FEF7CC
:102D6000BBFE5021884803F0DEFE0121864803F0B7
:102D7000DEFE81464946844803F0D3FE00BF824808
:102D800003F077FE0028FADADBE3FFE7012C7DD1C0
:102D90007B48401C02F04AFE7A48401C02F046FE86
:102DA0007848401C02F042FE4FF00110FEF7A2FCF2
:102DB0007748FEF79FFC01217648FEF7E7FC0221E9
:102DC0007448FEF7E3FC02F0A9FE824604EB4400DF
:102DD0006A4901EBC000806804EB4401DFF89CC144
:102DE0000CEBC101C968084304EB44010CEBC101C1
:102DF000096940EA010304EB4400614601EBC000AD
:102E000051464268644803F04CFE5E48093002F0C7
:102E10000DFE012210216148FEF78CFB0C230122DC
:102E200010215E48FEF7A0FB04EB4400534901EB80
:102E3000C0004078022819D152480A3002F0F6FD4D
:102E4000EF2210215548FEF7B0FC012211465448EC
:102E5000FEF770FB0C23012211465148FEF784FB5C
:102E6000FE2201214E48FEF7A0FC04E0102211468C
:102E70004A48FEF79AFC4B490620FEF739F906202E
:102E8000FDF7CCFE1620FEF7E5FD00E017E060211F
:102E90001620FEF721FE50213F4803F044FE012199
:102EA0003D4803F044FE814649463B4803F039FE65
:102EB00000BF394803F0DDFD0028FADA41E3022CB7
:102EC00078D12F48801C02F0B1FD2E4802F0AEFDF3
:102ED0002C4802F0ABFD41F60100FEF70BFC41F679
:102EE0000140FEF707FC40214FF04020FEF74EFC6A
:102EF00080214FF04020FEF749FC02F00FFE824691
:102F000004EB44001D4901EBC000806804EB440160
:102F1000DFF868C00CEBC101C968084304EB440149
:102F20000CEBC101096940EA010304EB440061466E
:102F300001EBC000514642681B4803F0B2FD04EBB0
:102F400044000E4901EBC0004078022813D10D481F
:102F5000401D02F06BFD012210211448FEF7EAFA31
:102F60000C23012210211148FEF7FEFAEF22102156
:102F70000E48FEF71AFC0E4921201CE0BC00002080
:102F8000001800F0000800F000C00040C927000051
:102F9000010401000050004000D000400010064035
:102FA000002006403528000000E0004000500240AC
:102FB000A12800001FE0FEF79BF82120FDF72EFE60
:102FC0003120FEF747FD60213120FEF785FD5021BD
:102FD000FE4803F0A8FD0121FC4803F0A8FD81464E
:102FE0004946FA4803F09DFD00BFF84803F041FD53
:102FF0000028FADAA5E2032C7ED1F54802F016FD8E
:10300000F44802F013FDF34802F010FD41F2010014
:10301000FEF770FB41F20140FEF76CFB10214FF010
:103020004020FEF7B3FB20214FF04020FEF7AEFB1F
:1030300002F074FD824604EB4400E74901EBC00056
:10304000806804EB4401DFF890C30CEBC101C96850
:10305000084304EB44010CEBC101096940EA010398
:1030600004EB4400614601EBC00051464268DB4876
:1030700003F017FD04EB4400D74901EBC000407892
:10308000022816D1D34802F0D1FC012202214FF0D0
:103090004020FEF74FFA4FF48473012202214FF0D3
:1030A0004020FEF761FAFD2202214FF04020FEF79A
:1030B0007CFBCB493820FEF71BF83820FDF7AEFD2E
:1030C0004820FEF7C7FC60214820FEF705FD50218F
:1030D000C24803F028FD0121C04803F028FD8146C5
:1030E0004946BE4803F01DFD00BFBC4803F0C1FCCB
:1030F0000028FADA25E2FFE7042C7DD1B448401C11
:1031000002F094FCB34802F091FCB24802F08EFC4D
:1031100040F60100FEF7EEFA40F60140FEF7EAFA4B
:1031200004214FF04020FEF731FB08214FF04020F2
:10313000FEF72CFB02F0F2FC824604EB4400A649A9
:1031400001EBC000806804EB4401DFF88CC20CEB9B
:10315000C101C968084304EB44010CEBC1010969D2
:1031600040EA010304EB4400614601EBC000514614
:1031700042689C4803F095FC04EB4400964901EB3F
:10318000C0004078022816D1924802F04FFC01227C
:1031900002214FF04020FEF7CDF94FF48473012255
:1031A00002214FF04020FEF7DFF9FD2202214FF00F
:1031B0004020FEF7FAFA8C493920FDF799FF3920B3
:1031C000FDF72CFD4920FEF745FC60214920FEF764
:1031D00083FC5021834803F0A6FC0121814803F0C1
:1031E000A6FC814649467F4803F09BFC00BF7D4812
:1031F00003F03FFC002800E001E0F8DAA1E1052C33
:103200007DD17348801C02F011FC7248801C02F0D2
:103210000DFC7048801C02F009FC7448FEF76AFA45
:103220007348FEF767FA40217248FEF7AFFA802133
:103230007048FEF7ABFA02F071FC824604EB4400E2
:10324000654901EBC000806804EB4401DFF888C1E8
:103250000CEBC101C968084304EB44010CEBC1014C
:10326000096940EA010304EB4400614601EBC00038
:1032700051464268604803F014FC04EB4400564990
:1032800001EBC0004078022816D1524802F0CEFB74
:10329000012202214FF04020FEF74CF94FF48473D5
:1032A000012202214FF04020FEF75EF9FD220221AB
:1032B0004FF04020FEF779FA50493A20FDF718FF09
:1032C0003A20FDF7ABFC4A20FEF7C4FB60214A2000
:1032D000FEF702FC5021484803F025FC0121464836
:1032E00003F025FC81464946434803F01AFC00BF21
:1032F000414803F0BEFB0028FADA22E1FFE7062C82
:1033000062D13348C01C02F091FB32480D3002F00C
:103310008DFB30480D3002F089FB3948FEF7EAF9A1
:103320003848FEF7E7F901213748FEF72FFA022166
:103330003548FEF72BFA02F0F1FB824604EB44001D
:10334000254901EBC000806804EB4401DFF888C028
:103350000CEBC101C968084304EB44010CEBC1014B
:10336000096940EA010304EB4400614601EBC00037
:1033700051464268254803F094FB04EB440016498B
:1033800001EBC0004078022816D1124802F04EFB33
:10339000012202214FF04020FEF7CCF84FF4847355
:1033A000012202214FF04020FEF7DEF8FD2202212B
:1033B0004FF04020FEF7F9F915493B20FDF798FE44
:1033C0003B20FDF72BFC25E03FE0000000E0004043
:1033D000031800F0000800F0BC00002000F00040DE
:1033E0000D290000000001407929000001180200A9
:1033F000011C02000060004000100140E5290000AF
:1034000001000D0001040D000050064000200140A5
:10341000512A00004B20FEF71DFB60214B20FEF7D8
:103420005BFB50214B4803F07EFB0121494803F030
:103430007EFB81464946474803F073FB00BF454881
:1034400003F017FB0028FADA7BE0072C79D1424819
:1034500002F0ECFA414802F0E9FA404802F0E6FADC
:103460003F48FEF747F93F48FEF744F910213E4830
:10347000FEF78CF920213C48FEF788F902F04EFB5C
:10348000824604EB4400394901EBC000806804EB3C
:103490004401DFF8D8C00CEBC101C968084304EB54
:1034A00044010CEBC101096940EA010304EB44004B
:1034B000614601EBC000514642682D4803F0F1FA25
:1034C00004EB4400294901EBC0004078022817D1E1
:1034D0002248801E02F0AAFA012202214FF0402069
:1034E000FEF728F84FF48473012202214FF04020A8
:1034F000FEF73AF8FD2202214FF04020FEF755F981
:103500001C493C20FDF7F4FD3C20FDF787FB4C20D7
:10351000FEF7A0FA60214C20FEF7DEFA5021144895
:1035200003F001FB0121124803F001FB81464946EB
:103530000F4803F0F6FA00BF0D4803F09AFA00288E
:10354000FADA012004EB4401084A02F831000020B5
:10355000FFF7F6BA00200140071800F0020800F05B
:10356000011002000114020000600040BC000020B5
:1035700000300140BD2A00002DE9F04104460E460E
:1035800017460025A846082C02DB681EBDE8F0811E
:1035900004EB4400C44911F83000012802D04FF078
:1035A000FF30F3E700BF04EB4400BF4901EBC0006C
:1035B000007D0128F7D0012004EB4401BA4A02EB58
:1035C000C1010875FCF78EFE804654BB04EB440035
:1035D000B54901EBC0004078022805D1022211460E
:1035E0004FF04020FEF7E1F804E0715DAF4803F0D2
:1035F0004AFA6D1CBD42F8D300BFAC4803F034FA60
:103600000028FAD104EB4400A74901EBC000407840
:10361000022805D1FD2202214FF04020FEF7C5F817
:1036200035E1012C28D104EB44009F4901EBC00097
:103630004078022804D1012211469D48FEF7B5F8D2
:1036400004E0715D9B4803F01EFA6D1CBD42F8D387
:1036500000BF984803F008FA0028FAD104EB4400B0
:10366000914901EBC00040780228D9D1FE22012106
:103670008F48FEF79AF80AE1022C28D104EB4400A7
:10368000894901EBC0004078022804D1102211467C
:103690008948FEF78AF804E0715D884803F0F3F981
:1036A0006D1CBD42F8D300BF844803F0DDF900284B
:1036B000FAD104EB44007C4901EBC00040780228B9
:1036C000AED1EF2210217C48FEF76FF8DFE0032C2B
:1036D0002AD104EB4400744901EBC0004078022871
:1036E00005D1022211464FF04020FEF75EF804E0BB
:1036F000715D734803F0C7F96D1CBD42F8D300BF7C
:103700006F4803F0B1F90028FAD104EB4400664990
:1037100001EBC00040780228ADD1FD2202214FF01C
:103720004020FEF742F8B2E0042C2AD104EB44001A
:103730005D4901EBC0004078022805D10222114604
:103740004FF04020FEF731F804E0715D5D4803F072
:103750009AF96D1CBD42F8D300BF5A4803F084F9B2
:103760000028FAD104EB44004F4901EBC000407837
:10377000022805D1FD2202214FF04020FEF715F866
:1037800085E0052C2AD104EB4400474901EBC00039
:103790004078022805D1022211464FF04020FEF762
:1037A00004F804E0715D484803F06DF96D1CBD42FA
:1037B000F8D300BF444803F057F90028FAD104EBCE
:1037C0004400394901EBC000407802285FD1FD2256
:1037D00002214FF04020FDF7E8FF58E0062C2AD1E7
:1037E00004EB4400304901EBC0004078022805D1C9
:1037F000022211464FF04020FDF7D7FF04E0715D33
:10380000324803F040F96D1CBD42F8D300BF2F4889
:1038100003F02AF90028FAD104EB4400224901EB15
:10382000C0004078022832D1FD2202214FF0402012
:10383000FDF7BBFF2BE0072C29D104EB44001A490C
:1038400001EBC0004078022805D1022211464FF05A
:103850004020FDF7AAFF04E0715D1D4803F013F955
:103860006D1CBD42F8D300BF194803F0FDF80028D5
:10387000FAD104EB44000C4901EBC0004078022867
:1038800005D1FD2202214FF04020FDF78EFF40467A
:10389000FCF72CFD002004EB4401034A02EBC101BC
:1038A000087500BF72E60000BC00002000C00040A8
:1038B0000020064000D000400050024000E00040E0
:1038C00000F00040000001400010014000200140D5
:1038D0000030014010B50246082A00DA11B94FF055
:1038E000FF3010BD02EB42001E4B13F830000128E0
:1038F00002D04FF0FF30F4E700BF02EB4200194B5B
:1039000003EBC000407D0128F7D0012002EB420309
:10391000144C04EBC3035875082A1DD2DFE802F0EB
:1039200004070A0D101316190F48016017E00F481D
:10393000016014E00E48016011E00E4801600EE0E5
:103940000D4801600BE00D48016008E00C48016083
:1039500005E00C48016002E04FF0FF30C1E700BF16
:103960000020BEE7BC0000209C000020A00000203A
:10397000A4000020A8000020AC000020B00000201F
:10398000B4000020B800002010B54FF0804003F0D4
:10399000E7F802F0C3F8044621464FF0804003F0F8
:1039A000D8F84FF0804003F0D0F810BD0020014956
:1039B000087070477C01002010B54FF0704002F095
:1039C00035F82220FEF746F84FF0804003F0C8F8A3
:1039D00002F0A4F8044621464FF0804003F0B9F805
:1039E0004FF0804003F0B7F84FF0804003F0ADF89F
:1039F00005491220FDF77CFB1220FDF70FF94FF06F
:103A0000804003F09AF810BD0D3A000010B500F0A8
:103A100097F90C480078401C0A490870084600785D
:103A20001E2802DD0120084908700748007828B9DF
:103A30004FF0804003F086F8FFF7A6FF00F09AF9F8
:103A400010BD00007C0100207D0100200120014903
:103A5000087070477D01002030B505460C462246AF
:103A60000021284600F026F830BD00000D480E4920
:103A700001600146416000218160C16001614161D6
:103A80008161C16101620163C16241620749816371
:103A9000C1634FF48061016441640146044A1160CE
:103AA00070470000080200204845415050020020A5
:103AB000040000202DE9F04103460C4617460FB9DB
:103AC000BDE8F08103B9FBE70025002202E02D02EA
:103AD0002543521C042AFAD3384603F0030C194636
:103AE000BCF1000F08D0624603E001F8014B401E14
:103AF000521C08B1042AF8D30E4601E020C6001F6C
:103B00000428FBD2314602E001F8014B401E002898
:103B1000FAD100BFD4E700001D481E481E481F48C8
:103B20001F4820482048214821482248224823484D
:103B3000234824482448254825482648264827481D
:103B4000274828482848294829482A482A482B48ED
:103B50002B482C482C482D482D482E482E482F48BD
:103B60002F4830483048314831483248324833488D
:103B7000334834483448354835483648364837485D
:103B80003748384838483948394800BF704700003E
:103B90005C96000060960000669600006896000043
:103BA000649600006A9600006C9600006E96000015
:103BB00070960000729600007496000076960000E1
:103BC000789600007A9600007C9600007E960000B1
:103BD0008096000082960000849600008696000081
:103BE000889600008A9600008C9600008E96000051
:103BF0009096000092960000949600009696000021
:103C0000989600009A9600009C9600009E960000F0
:103C1000A0960000A2960000A4960000A6960000C0
:103C2000A8960000AA960000AC960000AE96000090
:103C3000B2960000B4960000B6960000B896000058
:103C4000001C002080200020BC960000BE960000D2
:103C5000C0960000C2960000C4960000C696000000
:103C6000C8960000CA960000CC960000BA960000E4
:103C7000CE9600002DE9F04105460E461446002779
:103C80001148007818B112202070BDE8F081287822
:103C9000012808D0022807D0032802D0042804D124
:103CA00000E000BF00BF00BF02E001202070ECE791
:103CB00000BFFCF717FB07466E613846FCF716FBA2
:103CC0000020207000BFE0E72500002010B500F0C4
:103CD00019F801F07FF801F0ABF801F0CBF801F032
:103CE00049F801F009F801F05FF901F089F901F0F4
:103CF00001F901F027F900F0CFFD00F01FF8FFF700
:103D00000BFF10BD0948802102E0491E002204C0BB
:103D10000029FAD1064A074B1A601A46126822F0A7
:103D200007021A600022044B1A807047C02000204E
:103D3000C0220020700000207400002070470000A6
:103D400010B50024FCF7CEFA044608480078012894
:103D500008D107480078FF2804D205480078401CA5
:103D6000034908702046FCF7C1FA10BD320000205C
:103D70002500002010B500241A480078012830D111
:103D8000FCF7B0FA04461848007820B116480078CD
:103D9000401E1549087014480078F8B91348007897
:103DA000E0B901F08FF912481249097850F8210062
:103DB000114908600F4800781049097888420DD0F1
:103DC0000D480068C06B401C0B490968C8630C486B
:103DD0000068401C0A490860FCF7A4FA2046FCF77A
:103DE00085FA10BD320000202500002026000020AA
:103DF000981200202800002040000020270000200A
:103E00000C00002010B500240B480078012811D1C7
:103E1000FCF768FA04460948007840B90848007879
:103E2000FF2804D206480078401C05490870204647
:103E3000FCF75CFA10BD00003200002025000020D5
:103E40002600002010B5002413480078012821D155
:103E5000FCF748FA044611480078C0B910480078C9
:103E600088B10F480078401E0D4908700846007858
:103E700028B92046FCF73AFA01F0EAF80AE02046B1
:103E8000FCF734FA06E02046FCF730FA02E0204660
:103E9000FCF72CFA10BD00003200002025000020A5
:103EA0002600002070B5054600261048007808B1AD
:103EB000002070BDFCF716FA06460D48046800683D
:103EC00020B10B4800684068094908603046FCF79B
:103ED0000DFA4CB10320207025810020606005A000
:103EE0006061204600F0FAFE2046E2E7250000204F
:103EF000100000203F0000002DE9F04105460E466D
:103F0000144600272878032803D001202070BDE83C
:103F1000F0813248007810B102202070F7E7304875
:103F2000007810B10D202070F1E7FCF7DBF90746AF
:103F3000288940B12889401E28813846FCF7D6F9E7
:103F400000202070E3E72748006890F8340040F034
:103F500001002449096881F83400002021490968DA
:103F600081F835001F4800680663284600F078FE97
:103F70003846FCF7BBF901F06BF8FCF7B3F90746DC
:103F80001848006890F8350020B1012809D00228AF
:103F900006D102E0002020700BE00E20207008E027
:103FA00000BF29460F48006800F026FE0A20207056
:103FB00000BF00BF00200B49096881F8340009499F
:103FC000096881F8350007490968C8610549096829
:103FD00008623846FCF78AF900BF98E72500002000
:103FE000260000203800002070B504460025207807
:103FF000032801D0012070BDFCF774F90546A07AB2
:1040000060B1002301221946204600F0ADFD28468C
:10401000FCF76CF901F01CF80020ECE720894FF662
:10402000FF71884207D22089401C20812846FCF776
:104030005DF90020DFE72846FCF758F93320DAE77E
:1040400010B50B48007890B901F03CF809480078A9
:104050000949087009480749097850F821000849BA
:1040600008600846006807490860FCF742F910BD7F
:104070003200002028000020270000209812002095
:10408000400000203800002010B50024022000F07D
:1040900035FBFCF727F9044600200B490860204651
:1040A000FCF724F9642000F029FBFCF71BF9044617
:1040B0000548006805490860012005490870204648
:1040C000FCF714F910BD0000340000201C00002093
:1040D0002400002010B504462046FCF791FD10BDD9
:1040E0002DE9F04F85B081468A4693461C46DDE9AE
:1040F0000F78129D00200390FCF7F4F803902348FA
:10410000007830B10398FCF7F1F83C2005B0BDE829
:10411000F08F1F4850F8240088BB01201C4941F84B
:1041200024000398FCF7E2F82A464146384601F09D
:104130000DF92B465A465146484600F073F9049053
:104140001198CDE9008002953A4620460E9B0499CD
:1041500000F0CEFF064636B90E48007801280CD193
:1041600000F076FF09E0FCF7BDF803900020084955
:1041700041F824000398FCF7B9F83046C6E7FFE79A
:104180000398FCF7B3F82820C0E7000025000020C2
:10419000981200203200002010B504462046FCF79B
:1041A00030FD10BD2DE9F041054600274A48007852
:1041B00010B14020BDE8F0813F2D01D13E20F9E74C
:1041C000FCF790F80746FF2D03D14448006890F8AB
:1041D0003650434850F8254024B93846FCF786F855
:1041E0004320E7E7012C04D13846FCF77FF83D2057
:1041F000E0E714F8380F3B49085C61788843217880
:10420000384A505414F838091146085C30B994F80B
:104210003A1035480078884333490870E06918B18E
:104220002046E16900F0E8FC206A18B12046216AC6
:1042300000F0F9FCA66A16B1304600F089FD0020B6
:10424000206384F8340084F8350028480078FF287B
:1042500004D226480078401C244908703846FCF7F0
:1042600045F800F07FFCFCF73DF807461F48007852
:1042700020B11E480078401E1C490870204600F0FE
:1042800041F81B480078401E194908700020144965
:1042900041F82500A06930B900206169886115499D
:1042A0006069086005E0D4E905014861D4E90510BA
:1042B00088611148006860610F4804600FA02065A4
:1042C0003846FCF713F80E480078012801D100F0B9
:1042D000BFFE00206EE7000025000020380000200F
:1042E000981200202A00002029000020260000202B
:1042F00033000020440000203C0000203F0000006C
:104300003200002010B504462046FCF77BFC10BDAF
:1043100010B5FCF778FC10BD2DE9F04106460F46BC
:1043200014464FF000081548007818B1122020708C
:10433000BDE8F081FBF7D6FF8046FF2E03D1104881
:10434000006890F836600F4850F826502DB9404666
:10435000FBF7CCFF43202070EAE7012D05D1404652
:10436000FBF7C4FF43202070E2E72F654046FBF7D0
:10437000BDFF0020207000BFDAE70000250000200C
:10438000380000209812002010B504462046FCF7A3
:104390003BFC10BD10B5FCF738FC10BD2DE9F04713
:1043A00007460D464FF0000A002028606860FBF7C2
:1043B00099FF8246FF2F03D11848006890F83670A5
:1043C000174850F827402CB95046FBF78FFF432081
:1043D000BDE8F087012C04D15046FBF787FF43204E
:1043E000F6E7207C00F0010020B95046FBF77EFF85
:1043F0004520EDE70026D4F80C90D4F8088050460C
:10440000FBF774FF00E0761C58F8041B0029FAD073
:104410002E60A9EB060068600020D9E73800002074
:104420009812002070B50446101D20F007004FF0D0
:104430008076051F28462E60051F28462C60684E92
:10444000051F28462E604FF01236051F28462E60A5
:104450004FF00336051F28462E604FF00236051F29
:1044600028462E607610051F28462E60051F284618
:1044700029604FF01136051F28462E604FF0103688
:10448000051F28462E604FF00936051F28462E606E
:104490004FF00836051F28462E604FF00736051FDF
:1044A00028462E604FF00636051F28462E604FF036
:1044B0000536051F28462E604FF00436051F284696
:1044C0002E6003F00405002D7ED0F605051F28465A
:1044D0002E60444E051F28462E60434E051F284679
:1044E0002E60424E051F28462E60414E051F28466D
:1044F0002E60404E051F28462E603F4E051F284661
:104500002E603E4E051F28462E603D4E051F284654
:104510002E603C4E051F28462E603B4E051F284648
:104520002E603A4E051F28462E60394E051F28463C
:104530002E60384E051F28462E60374E051F284630
:104540002E60364E051F28462E604FF08346051F0D
:1045500028462E60324E051F28462E60314E051F1C
:1045600028462E60304E051F28462E602F4E051F10
:1045700028462E602E4E051F28462E602D4E051F04
:1045800028462E602C4E051F28462E604FF082468E
:10459000051F28462E60294E051F28462E60284EEE
:1045A000051F28462E60274E051F28462E604FF017
:1045B0008146051F28462E60234E051F28462E6083
:1045C0003602051F284600E009E02E604FF07E56B7
:1045D000051F28462E600026051F28462E6070BD48
:1045E000595200000000F8410000F0410000E8418D
:1045F0000000E0410000D8410000D0410000C84167
:104600000000C0410000B8410000B0410000A841D6
:104610000000A04100009841000090410000884146
:104620000000704100006041000050410000404126
:104630000000304100002041000010410000E04037
:104640000000C0400000A040000040402DE9F041C3
:1046500005464FF00008FBF745FE8046FF2D05D1CB
:104660002048006890F83650012608E01D48006890
:1046700090F83600A84201D1012600E000261A4831
:1046800050F825402CB94046FBF730FE4820BDE8E5
:10469000F081012C04D14046FBF728FE4320F6E7C9
:1046A00094F838701148C05D94F8391088430F4968
:1046B000C8550846C05D30B994F83A100C480078E7
:1046C00088430B49087094F8340040F0080084F8DF
:1046D00034004046FBF70AFE012E01D100F0B8FC81
:1046E0000020D4E738000020981200202A00002083
:1046F0002900002010B5FCF789FA10BD70B50546F9
:1047000000261748007800B170BD1648007800B147
:10471000FAE71DB3FBF7E6FD06461348006890F87C
:1047200038401248005D1049096891F839108843F3
:104730000E4908550846005D40B90B48006890F8DE
:104740003A100B4800788843094908700648006809
:1047500005633046FBF7CAFD00F07AFC00BFD3E7E3
:104760002500002026000020380000202A0000201C
:104770002900002070B5002600F072F8FBF7B2FDAA
:10478000064631480068401C2F4908603046FBF758
:10479000ADFD2E480078012853D12D48007820B176
:1047A000012804D0022809D103E001250BE00025EF
:1047B00009E0012501202649087004E001250020B8
:1047C0002349087000BF00BF05B970BD21480468C7
:1047D00033E0FBF787FD0646206B50B3206B401E8D
:1047E0002063206B28BB94F8340000F0370040B100
:1047F00014F8340F00F0C800207001206070343CC1
:1048000002E0002084F8350094F8340000F008003D
:1048100078B93834A0781049097808430E490870EF
:1048200020780E49085C6178084314F838190B4A5F
:10483000505464693046FBF759FD94F836003F2820
:10484000C7D100BFC1E7000058000020320000209F
:104850004800002044000020290000202A000020F9
:1048600010B5FCF7D4F906480088401C04490880BC
:104870000846008818B10020088000F003F810BD39
:104880007400002010B503480068FFF7ADFB044634
:10489000204610BD68000020F8B54FF4207128486C
:1048A00000F078FB4021274800F074FB002514E05D
:1048B000681C86B205EB8500214901EBC00406EBBC
:1048C000860001EBC00764202070002084F82500DA
:1048D000E7601DA02062681C85B20F2DE8D305EBB0
:1048E0008500174901EBC00464202070002084F883
:1048F0002500E06014A020620020144908601449DB
:1049000008801020134908800D48134908600120D1
:10491000FFF7C8FA114908600020FFF7C3FA1049F1
:1049200008606A460FA10D480068FFF7A3F96A46C0
:1049300011A10B480068FFF79DF900F027F8F8BDBA
:10494000001C0020802000203F00000060000020AC
:104950005E0000205C0000206C000020640000204D
:104960006800002075432F4F532D494920546D7224
:104970004C6F636B0000000075432F4F532D494966
:1049800020546D725369676E616C000000B587B08A
:104990000320002180220A4BCDE90132CDE903102A
:1049A0004FF6FD703D23074A00900748FFF798FB3C
:1049B00006AA06A13D20FFF7AFFC07B000BD00002E
:1049C000801E00207C200020494A000075432F4FA4
:1049D000532D494920546D720000000070B50B46FC
:1049E000032580F82550012B05D1154EC569366881
:1049F000354445610CE085692DB9114EC5693668AD
:104A00003544456104E00E4E85693668354445619C
:104A1000057D05F007040B4D05EBC4010D682DB9AC
:104A200008600025C56001258D8006E00A680860E1
:104A3000C26010618D886D1C8D800025056170BD80
:104A4000600000208020002008B500BF00BF6A463B
:104A500000211A480068FFF74FFAFFF7D3F918480A
:104A60000068401C164908600846007800F00708F6
:104A7000144800EBC8073C681AE0E6681049606912
:104A80000968884213D1204600F01EF894F82400EB
:104A9000022804D101212046FFF7A0FF02E00220F6
:104AA00084F82500656815B12046A168A8473446FA
:104AB000002CE2D1FFF7C6F9C9E70000680000202A
:104AC000600000208020002030B5057D05F007043F
:104AD0000D4D05EBC4031D68854205D1C168196001
:104AE00039B100250D6104E00169C268CA6002B1F4
:104AF0001161012580F825500025C56005619D885C
:104B00006D1E9D8030BD00008020002010B5FBF799
:104B1000E9FB044606480078401C05490870204619
:104B2000FBF7E4FBFFF726FEFFF724F910BD0000BA
:104B30002500002001464A1E4FF0E0235A61084A32
:104B4000106820F07F4000BF10601A46126942F0E2
:104B500005021A611A46126942F002021A61704790
:104B600020ED00E0704700002DE9F04F05460F46AC
:104B700090469946A87A1C490E5C05F10B00805DB1
:104B800011F800B00BEBC60000F0FF0A174850F810
:104B90002A4000202434E0602760207C20EA0800BE
:104BA000207484F81190207C243C00F0080068B93F
:104BB00094F83A000E49097808430D4908700D48E9
:104BC000805D94F8391008430A49885529462046E3
:104BD00000F012F8206A20B12046216A00F023F884
:104BE000E5615046BDE8F08F5C950000981200200A
:104BF000290000202A00002010B590F8382001F18B
:104C00000B039B5C90F83940A34301F10B04A354C0
:104C100023469B5C23B98B7A90F83A40A3438B726E
:104C20000023C36110BDF0B5024612F8384F9578E5
:104C30005678383A0B4618680FE000F10B073F5DD5
:104C4000B74300F10B0C0CF8047067463F5D17B9D1
:104C5000877AAF4387721B1D18680028EDD1F0BD1D
:104C600010B51B4A1268D061194A126892F83830A0
:104C700000F10B02D25C164B1B6893F839301A43D3
:104C8000134B1B6893F8384000F10B031A55827AD6
:104C90000F4B1B6893F83A301A4382720C4A126821
:104CA00092F838100B4A525C094B1B6893F8393064
:104CB0009A43084B5A541A46525C42B9044A126845
:104CC00092F83A30044A12789A43034B1A7010BD96
:104CD000380000202A000020290000200146002280
:104CE0008A72002005E0002301F10B021354421CDC
:104CF000D0B20828F7D370472DE9F041A021114820
:104D000000F048F900250DE0681C86B20D4800EB64
:104D1000051400EB06170020207067600AA0E06011
:104D2000681C85B2092DEFD3064800EB051400205E
:104D30002070606004A0E060024804490860BDE89B
:104D4000F0810000F80D00203F000000140000205A
:104D500030B501464A6808682AB9CC68606028B155
:104D60000025456002E0106000B142608B680025BC
:104D70009D6230BD70B54FF4BD61134800F00AF973
:104D8000002411E0601C85B204EB44000E4901EBE5
:104D9000C00305EB450001EBC006002018705E6003
:104DA0000AA05861601C84B23E2CEBD304EB440093
:104DB000054901EBC00300201870586003A058613A
:104DC00008460349086070BD100800203F0000003D
:104DD0001000002000200B4908600B4908700B49A7
:104DE00008700B4908700B4908700B4908600B49A3
:104DF00008600B4908600B4908600B4908700B49B3
:104E00000870704758000020250000202600002070
:104E100033000020320000200C000020340000206D
:104E2000200000201C00002024000020540000204E
:104E300000210A4A1170002004E00021084A1154A0
:104E4000411CC8B20828F8D30021064A1170064A4E
:104E50001170064A1160064A11607047290000204F
:104E60002A00002027000020280000204000002009
:104E70003800002070B54FF4F261194800F08AF84C
:104E80004FF48071174800F085F8002413E0601C8F
:104E9000C5B204EB440000EBC400114901EBC003B0
:104EA00005EB450000EBC50001EBC0065E610EA0FE
:104EB0001865601CC4B2152CE9D304EB440000EB68
:104EC000C400074901EBC0030020586106A0186523
:104ED00000200649086002480549086070BD0000CE
:104EE00098130020981200203F000000440000208A
:104EF0003C00002000B587B00320002180220A4B2F
:104F0000CDE90132CDE903104FF6FF703F23074A88
:104F100000900748FFF7E4F806AA06A13F20FFF734
:104F2000FBF907B000BD000098100020941200208B
:104F30003152000075432F4F532D49492049646C6D
:104F40006500000000B587B00320002180220A4BD5
:104F5000CDE90132CDE903104FF6FE703E23074A3A
:104F600000900748FFF7BCF806AA06A13E20FFF70D
:104F7000D3F907B000BD0000980E00209410002067
:104F80007152000075432F4F532D494920537461CE
:104F90007400000004E0002200F8012B4A1E91B2C8
:104FA0000029F8D17047000070B578211148FFF74B
:104FB000F1FF00240EE004EB44000E4901EBC005B4
:104FC000601C00EB400001EBC00068600AA0686153
:104FD000601C84B2042CEED304EB4400054901EBC1
:104FE000C0050020686004A06861084603490860A5
:104FF00070BD0000281B00203F0000004C00002076
:105000002DE9F04160211048FFF7C4FF00240DE0B6
:10501000601C86B204EB44000B4901EBC00506EBB3
:10502000460001EBC0072F60601C84B2032CEFD355
:1050300004EB4400044901EBC00500202860084649
:1050400002490860BDE8F081A01B0020500000204C
:1050500010B50024FBF746F9044613480078F8B968
:1050600012480078E0B900F02DF81148114909788C
:1050700050F82100104908600E4800780F4909785F
:1050800088420DD00C480068C06B401C0A49096872
:10509000C8630B480068401C09490860FBF73DF9EC
:1050A0002046FBF723F910BD250000202600002034
:1050B0009812002028000020400000202700002037
:1050C0000C0000200649074A1278885C0649095CF2
:1050D000034A515C01EBC001044A117070470000A3
:1050E0005C950000290000202A00002028000020F4
:1050F0002DE9F84F05460F4690469946DDE90AAB83
:1051000000200090FBF7EEF8009042480468002C65
:105110007BD01C3454F8080C3E4908600098FBF71B
:10512000E5F844F81C7CA576002020766076606166
:1051300044F818BC44F810AC44F8148C0C9824F8CB
:105140000C0C24F80A9C0020E077E810207705F08A
:105150000700E076217F01208840A077E17E0120D2
:1051600088406077002020606060E060A06020627E
:10517000A0626062E062206327A060631C3C00269E
:1051800006E0002104F1540040F82610701CC6B25D
:10519000002EF6D02046FEF79DFFFBF7A3F8009007
:1051A0001E4840F825400098FBF7A0F82046FEF77F
:1051B000F3FFFBF797F80090194800686061002042
:1051C000A0611748006810B1154800688461144850
:1051D00004603834A07813490978084311490870ED
:1051E00020781149085C6178084314F838190E4A90
:1051F00050540E480078401C0C4908700098FBF78A
:1052000075F80020BDE8F88FFFE70098FBF76EF80F
:105210004220F7E73C0000203F00000098120020E9
:1052200044000020290000202A0000203300002034
:10523000002400BF00BFFBF755F80446054800688E
:10524000401C044908602046FBF750F8FFF760F85F
:10525000F1E700003400002010B504480068FFF7B3
:1052600093F8FF20FEF79EFF10BD000038000020DD
:1052700000BF00BF02E0C820FFF740FA1F480078D7
:105280000028F8D01E4800686421B0FBF1F01C49EA
:1052900008600846006828B900201A490870FF20F5
:1052A000FFF7D4F9FBF71EF804461548006864219F
:1052B0004843154908602046FBF718F800BFFBF784
:1052C00011F80446104800681049086000200E4993
:1052D00008602046FBF70AF80C480068084909688E
:1052E000B0FBF1F0C0F1640006490870FFF752F816
:1052F00000F00EF86420FFF701FAE0E72400002038
:105300001C00002018000020340000202000002095
:105310007CB5002514E069462846FFF73FF80646AD
:1053200066B9094850F8254044B1012C06D0D4E9AB
:10533000020100EB8100A0640198E064681CC5B222
:105340003F2DE8D97CBD00009812002002F0010337
:1053500043B102F002032BB102E0491E002308C052
:105360000029FAD17047000070B504460E48FCF7DA
:1053700021FA0546002D02DA4FF0FF3070BD0A48D1
:105380000089E0800848C079607107488079207101
:1053900005484079E07004480079A0700248C07860
:1053A00060700020EAE700005023002010B50120C3
:1053B00000F032FAFF2000F036FA10BD70B5054655
:1053C00001220021092000F0D4F9044624B910215B
:1053D000284600F079F90446FFF7E8FF0CB10120F8
:1053E00070BD0020FCE770B505464FF6FF7401E084
:1053F000601E84B2FF2000F016FAA84201D0002CF3
:10540000F6D10CB9FF2070BD0020FCE770B510216B
:105410001D48FBF728F81C48FFF7D0FF08B1002013
:1054200070BD1948007800F0C000402809D1164826
:10543000407A1549097A00EB0120401C84B2A5028C
:1054400020E01148407900F00F000F49897A00EB05
:10545000D1100D49497A01F0030100EB4100861C8F
:105460000948007A80110849C97900EB8100064992
:10547000897901F0030100EB8120441CA6F10900A9
:1054800004FA00F52846CBE7402300207CB508202D
:105490006E4B0022114600900320FCF747FE0020CF
:1054A00000F0BAF9002000F0A1F9002505E0FF2086
:1054B00000F0B9F90446681C85B2642DF7DB402082
:1054C00000F0B1F9002000F0AEF9002000F0ABF9D7
:1054D000002000F0A8F9002000F0A5F9952000F0C8
:1054E000A2F9142600BF95220021084600F041F9D8
:1054F0000446012C04D0301EA6F101018EB2F2D177
:10550000002053490870012C4AD187224FF4D571ED
:10551000082000F02EF9012847D1002506E0FF20E1
:1055200000F081F901A94855681C85B2042DF6DB0D
:105530009DF80600012879D19DF80700AA2875D1A9
:105540004FF6FE7600BF01220021372000F011F94E
:1055500001229107292000F00CF9044624B1301EE5
:10556000A6F101018EB2EED1002E5FD00122002102
:105570003A2000F0FEF8002858D1002506E0FF2070
:1055800000F051F901A94855681C85B2042DF6DBDD
:105590009DF8040000F0400018B106202C49087066
:1055A00044E004202A49087040E00122002137200D
:1055B00000F0DFF801220021292000F0DAF804468B
:1055C000012C17DC0220224908704FF6FE7600BF3E
:1055D00001220021372000F0CCF8012200212920EF
:1055E00000F0C7F80446BCB1301EA6F101018EB22E
:1055F000EED111E00120164908704FF6FE7600BF8B
:1056000001220021104600F0B4F8044624B1301EF7
:10561000A6F101018EB2F3D12EB101225102102068
:1056200000F0A7F810B1002009490870FFF7BEFE8E
:10563000012000F0DBF80648007808B100207CBDAE
:105640000CB12046FBE7AA20F9E7000040420F001A
:10565000800100202DE9F04106460F461546194805
:105660000078062800D07F02012D0CD10122394696
:10567000112000F07EF80446FCB96902304600F0C3
:1056800023F8044619E001223946122000F071F88F
:10569000044600BF4FF40071304600F015F8044690
:1056A00006F50076681EC0B2051E01D0002CF1D0B0
:1056B000012200210C2000F05CF8FFF777FE204665
:1056C000BDE8F0818001002070B504460D46FE2043
:1056D000FFF789FE08B1012070BD04E0FF2000F053
:1056E000A2F82070641C281EA5F101018DB2F5D12D
:1056F000FF2000F098F8FF2000F095F80020EBE77D
:1057000010B5002000F088F800F09AF808B90020E1
:1057100010BDFFF74BFE0120FAE72DE9F0410646E8
:105720000D4600F08DF8074617B10120BDE8F08165
:10573000284600F078F8FD2D19D0002404E0305DF3
:1057400000F071F8601C84B2B4F5007FF7DBFF2035
:1057500000F069F8FF2000F066F8FF2000F063F821
:10576000074607F01F00052801D00220DEE70020D1
:10577000DCE72DE9F04105460C4617464FF00008DE
:10578000FFF714FEFFF7BCFF10B1FF20BDE8F0816A
:1057900045F0400000F047F8200E00F044F8C4F354
:1057A000074000F040F8C4F3072000F03CF8E0B2F6
:1057B00000F039F8384600F036F80C2D02D1FF2001
:1057C00000F031F84FF01F0800BFFF2000F02BF869
:1057D000064606F0800030B1B8F10000A8F10101E2
:1057E00001F0FF08F1D13046D0E700001CB50446B7
:1057F00014B90748019001E006480190002001AB70
:105800000246014600900320FCF71EFE1CBD00006E
:10581000400D0300003FAB0110B5044621460320B4
:10582000FCF72CFC10BD38B50446002000906A46F9
:1058300021460320FCF726FF9DF8000038BD00003C
:1058400038B5002400BFFF20FFF7EDFF0546FF2D10
:1058500001D1002038BD641C6FF07F40B4FBF0F133
:1058600000FB114050B90820074B00221146009060
:105870000320FCF75BFC0020FFF7CEFF6FF07040C9
:105880008442E0D30120E5E740420F002DE9F041DA
:1058900006460F46154620480078062800D07F02AD
:1058A000012D0CD1012239461820FFF762FF044672
:1058B0006CBBFE213046FFF730FF044627E0164858
:1058C0000078012809D0012200213720FFF751FF7D
:1058D000012229461720FFF74CFF012239461920E3
:1058E000FFF747FF044694B900BFFC213046FFF79D
:1058F00014FF044606F50076681EC0B2051E01D0EE
:10590000002CF2D0FD210020FFF707FF0446FFF72F
:105910004DFD2046BDE8F081800100200146C868A9
:10592000C0F3001070472DE9F04F0C461D46DDE92D
:1059300009C815B94FF0000A01E04FF0040A5746B4
:105940004760B4FBFCF6002100BF891CB6FBF1FAEE
:10595000AAF10103FF2BF8D801614FEA827A4FEADE
:105960001A6902F0300249EA032A4AEA020AA8F157
:10597000010B4AEA0B070760BDE8F08F00BFC26861
:1059800002F00402002AFAD082680A6070470246D8
:10599000D06800F0040018B19068086001207047DA
:1059A0000020FCE700BFC26802F00202002AFAD021
:1059B00081607047416821F0020141607047416891
:1059C00041F002014160704770B504460D4616462D
:1059D0000CB9002070BD0DB90020FBE721462A4616
:1059E000002304E010780870491C521C5B1C21B194
:1059F0001AB1107808B1B342F4D301B10AB900204A
:105A0000E8E7B34201D2002008702046E2E710B573
:105A100002460B461146002001E0491C401C19B10A
:105A20000C780CB19842F8D310BD000010B50121DC
:105A3000C0F30722094B1A4402F0704242F0007290
:105A4000C0F30723054C2344C3F3130342EA431274
:105A5000C3B242EA8302116010BD000000E60F40AD
:105A60000146C1F307200B4A104400F0704040F09B
:105A70000070C1F30722074B1A44C2F3130240EA35
:105A80004210CAB240EA8200006808B101207047A3
:105A90000020FCE700EA0F4018B50121C0F30722FF
:105AA000184B1A4402F0704242F00072C0F3072310
:105AB000144C2344C3F3130342EA4312C3B242EA31
:105AC000830211600021009102E00099491C0091BD
:105AD00000991029F9D30021C0F30722094B1A4479
:105AE00002F0704242F00072C0F30723054C2344D9
:105AF000C3F3130342EA4312C3B242EA83021160C2
:105B000018BD000000E50F4002480349086000BFCF
:105B1000FEE700000400FA050CED00E00148006813
:105B20007047000008000020DDE00520FEF7E6FDDC
:105B30006D48007840B200F043FF002431E004EBF0
:105B4000C4006A4901EB8000408C022828D104EB94
:105B5000C401664A02EB810065A1FAF78FFC18B117
:105B600001206549086017E004EBC4015F4A02EBBD
:105B7000810062A1FAF782FC18B101206149086036
:105B80000AE004EBC401594A02EB81005EA1FAF776
:105B900075FC08B1FFF7B8FFE0B200F091FE02E03B
:105BA000641C0A2CCBDB00BF53480068012836D1A7
:105BB00000F0B6F8012000F0C5F8022000F0C2F8AD
:105BC000032000F0BFF8042000F0BCF8002000F033
:105BD000A7F84F490B20FCF705F84D49091D0A208D
:105BE000FCF700F84A4908310920FBF7FBFF484958
:105BF0000C310820FBF7F6FF454910310520FBF773
:105C0000F1FF434914310420FBF7ECFF0120404928
:105C1000091F086000F02CFC002037490860394853
:105C2000006801285FD180213A48FBF78BFD80286E
:105C300003D101203849087102E00020364908717B
:105C400040213448FBF77EFD402803D10120324932
:105C5000487102E000203049487120212D48FBF7AF
:105C600071FD202803D101202B49887102E000201A
:105C70002949887110212748FBF764FD102803D1BA
:105C800001202549C87102E000202349C871042180
:105C90002248FBF757FD042803D101201E49087252
:105CA00002E000201C49087208211C48FBF74AFD4D
:105CB000082803D101201849487202E00020164943
:105CC000487215490C310720FBF78CFF124910313F
:105CD0000620FBF787FF01200F49086000200949D3
:105CE000086000F0C5FB20E7A4010020702300201D
:105CF000414142420A000000A801002045454646B5
:105D00000A000000AC010020434344440A000000A4
:105D1000DC24002000300640082500200050004010
:105D200010B504462CB9EF2210210548FBF73DFDC4
:105D300004E0102211460248FBF737FD10BD0000B9
:105D40000020064030B52DED068B83B005460024BB
:105D5000012D7DD108221146FC48FBF726FD1022BB
:105D60001146FA48FBF721FD27E0641C02A9002038
:105D7000FBF738FF01A90120FBF734FF9DED020A74
:105D800038EE000AB0EE408A9DED010A38EE800A36
:105D9000F0EE408AB4F57A7F0CDD9FEDED0AC8EE97
:105DA000000AB0EE608A9FEDEA0AC8EE800AF0EEC3
:105DB000608A03E00120FEF7A1FCD6E700BFF722CE
:105DC0000821E248FBF7F1FCEF221021DF48FBF746
:105DD000ECFC38EE680A10EE101A0846FAF767FB7A
:105DE00041EC1A0BB0EE4A0AF0EE6A0A00F0DCFE53
:105DF000B0EE409AF0EE609A9FEDD60B53EC102B6C
:105E000051EC190BFAF766FB09D20020D34981F84F
:105E10002C009FEDD30A084680ED070A0BE238EE0E
:105E2000680AB5EEC00AF1EE10FA12DD88EE280A13
:105E3000F3EE040A20EE200ADFEDC50A80EE201AF8
:105E4000C64880ED071A0120C44981F82C00F2E110
:105E500011E088EE880AF3EE040A20EE200ADFED56
:105E6000BC0A80EE201ABD4880ED071A0220BB490B
:105E700081F82C00DFE1022D7ED102221146B348C9
:105E8000FBF793FC04221146B048FBF78EFC27E099
:105E9000641C02A90220FBF7A5FE01A90320FBF761
:105EA000A1FE9DED020A38EE000AB0EE408A9DED9B
:105EB000010A38EE800AF0EE408AB4F57A7F0CDDF4
:105EC0009FEDA30AC8EE000AB0EE608A9FEDA00A1B
:105ED000C8EE800AF0EE608A03E00120FEF70EFCB7
:105EE000D6E700BFFD2202219848FBF75EFCFB22AB
:105EF00004219648FBF759FC38EE680A10EE101A98
:105F00000846FAF7D4FA41EC1A0BB0EE4A0AF0EE62
:105F10006A0A00F049FEB0EE409AF0EE609A9FEDFA
:105F20008D0B53EC102B51EC190BFAF7D3FA09D265
:105F300000208A4981F82D009FED890A084680EDEE
:105F4000080A78E138EE680AB5EEC00AF1EE10FAF8
:105F500017DD9DED020A9DED011AC0EE010AB2EEB9
:105F6000050A20EE800ADFED7A0A80EE201A7B48CF
:105F700080ED081A012000E019E0784981F82D0031
:105F800059E19DED010ADDED020A80EE201AB2EE24
:105F9000050A21EE000ADFED6E0A80EE201A6F4836
:105FA00080ED081A02206D4981F82D0043E1032D90
:105FB0007ED1202211466B48FBF7F7FB01221146E8
:105FC0006248FBF7F2FB27E0641C02A91020FBF7F4
:105FD00009FE01A91120FBF705FE9DED020A38EE2E
:105FE000000AB0EE408A9DED010A38EE800AF0EE1C
:105FF000408AB4F57A7F0CDD9FED550AC8EE000AA1
:10600000B0EE608A9FED520AC8EE800AF0EE608A18
:1060100003E00120FEF772FBD6E700BFDF2220215C
:106020005048FBF7C2FBFE2201214848FBF7BDFBAD
:1060300038EE680A10EE101A0846FAF738FA41EC02
:106040001A0BB0EE4A0AF0EE6A0A00F0ADFDB0EEAF
:10605000409AF0EE609A9FED3F0B53EC102B51EC01
:10606000190BFAF737FA09D200203C4981F82E00C3
:106070009FED3B0A084680ED090ADCE038EE680A2D
:10608000B5EEC00AF1EE10FA17DD9DED020ADDED66
:10609000010A80EE201AB2EE060A21EE000ADFEDB8
:1060A0002C0A80EE201A2D4880ED091A012000E00C
:1060B00019E02A4981F82E00BDE09DED010ADDEDD1
:1060C000020A80EE201AB2EE060A21EE000ADFED87
:1060D000200A80EE201A214880ED091A02201F496B
:1060E00081F82E00A7E0042D72D1082211461D4828
:1060F000FBF75BFB102211461A48FBF756FB36E014
:10610000641C02A91220FBF76DFD01A91320FBF707
:1061100069FD9DED020A38EE000AB0EE408A9DED61
:10612000010A38EE800AF0EE408AB4F57A7F1BDD72
:106130009FED070AC8EE000AB0EE608A9FED040AE0
:10614000C8EE800AF0EE608A12E0000000400640CF
:1061500000007A440000000000407F40D824002066
:1061600000000000005006400120FEF7C7FAC7E714
:1061700000BFF72208213248FBF717FBEF2210215E
:106180002F48FBF712FB38EE680A10EE101A08468B
:10619000FAF78DF941EC1A0BB0EE4A0AF0EE6A0AF2
:1061A00000F002FDB0EE409AF0EE609A1FED170B82
:1061B00053EC102B51EC190BFAF78CF909D2002093
:1061C000204981F82F001FED1A0A084680ED0A0ABF
:1061D00031E038EE680AB5EEC00AF1EE10FA15DDCE
:1061E0009DED020ADDED010A80EE201AB2EE080AEA
:1061F00021EE000A5FED2A0A80EE201A114880ED98
:106200000A1A01200F4981F82F0014E09DED010AC0
:10621000DDED020A80EE201AB2EE080A21EE000A35
:106220005FED350A80EE201A064880ED0A1A02203A
:10623000044981F82F0003B0BDEC068B30BD00008F
:1062400000500640D824002008B5FBF759FD7E48D1
:10625000FFF7ECFB012210217C48FBF76BF90C23C4
:10626000012210217948FBF77FF9EF2210217748AE
:10627000FBF79BFA7448801CFFF7D8FB012208212A
:106280007348FBF757F90C23012208217048FBF7EC
:106290006BF9F72208216E48FBF787FA6A48801CE1
:1062A000FFF7C4FB012210216948FBF743F90C23D7
:1062B000012210216648FBF757F9EF2210216448AC
:1062C000FBF773FA6048801CFFF7B0FB0122022144
:1062D0005F48FBF72FF90C23012202215C48FBF7F2
:1062E00043F9FD2202215A48FBF75FFA5648801C09
:1062F000FFF79CFB012204215548FBF71BF90C23F7
:10630000012204215248FBF72FF9FB2204215048B7
:10631000FBF74BFA4C48C01CFFF788FB01222021F9
:106320004C48FBF707F90C23012220214948FBF7D1
:106330001BF9DF2220214748FBF737FA4248801C2F
:10634000FFF774FB012211464148FBF7F3F80C23D9
:10635000012211463E48FBF707F9FE2201213C4885
:10636000FBF723FA3848C01CFFF760FB0122082125
:106370003848FBF7DFF80C23012208213548FBF7EA
:10638000F3F8F72208213348FBF70FFA2E48C01C18
:10639000FFF74CFB012210212E48FBF7CBF80C2312
:1063A000012210212B48FBF7DFF8EF2210212948AA
:1063B000FBF7FBF92448401CFFF738FB0022802143
:1063C0002548FBF7B7F82048401CFFF72FFB0022B9
:1063D00040212148FBF7AEF81B48401CFFF726FB85
:1063E000002220211C48FBF7A5F81748401CFFF7A6
:1063F0001DFB002210211848FBF79CF812480938B1
:10640000FFF714FB002204211448FBF793F80E4811
:106410000938FFF70BFB002208211048FBF78AF828
:106420000020012308224FF4165100900320FCF7AE
:106430007BFB0B490320FDF74DFA0AA000F0DEFAC2
:106440000A49086008BD00000A0800F00020064064
:10645000004006400050064000300640005000401A
:10646000716600005461736B44706300A4010020E6
:1064700010B52DED108B9AB07048006801287CD1C2
:106480006E4890ED0A0A10EE101A0846FAF70FF857
:1064900041EC180B694890ED090A10EE101A0846F5
:1064A000FAF705F841EC190B644890ED080A10EE74
:1064B000101A0846F9F7FBFF41EC1A0B5F4890ED04
:1064C000070A10EE101A0846F9F7F1FF41EC1B0B12
:1064D0005A4890ED060A10EE101A0846F9F7E7FF41
:1064E00041EC1C0B554890ED050A10EE101A0846B9
:1064F000F9F7DDFF41EC1D0B504890ED040A10EE5A
:10650000101A0846F9F7D3FF41EC1E0B4B4890EDEB
:10651000030A10EE101A0846F9F7C9FF41EC1F0BE9
:10652000464890ED020A10EE101A0846F9F7BFFF30
:10653000CDE91801414890ED010A10EE101A084605
:10654000F9F7B5FFCDE916013C4890F82F003B491B
:1065500091F82E10394A92F82D20384B93F82C30B0
:10656000CDE91232CDE914108DED108B8DED0E9B1F
:106570008DED0CAB8DED0ABB00E01FE08DED08CB7F
:106580008DED06DB8DED04EB8DED02FB9DED180B23
:106590008DED000B9DED160B53EC102B284929486F
:1065A00000F0EEFA2748F9F77BFF0446224625491A
:1065B0000320FCF7E1FF0020204908602248006822
:1065C000012836D1204890ED040A10EE101A084632
:1065D000F9F76DFF41EC180B1B4890ED030A10EE24
:1065E000101A0846F9F763FF41EC190B8DED068B85
:1065F0008DED049B1448407A1349097A124AD279E6
:10660000114B9B79CDE90032CDE902100E48437958
:1066100002790EA10B4800F0B3FA0A48F9F740FFDF
:106620000446224607490320FCF7A6FF002006493E
:1066300008601AB0BDEC108B10BD0000D8240020FB
:106640003C9B00001C2500200825002045454646AF
:106650002C25642C25642C25642C25642C25642C85
:1066600025642C25302E32662C25302E32660A0009
:1066700030B5014600203AE000EBC002414B03EB8D
:106680008202528C012A31D100EBC00203EB82025C
:1066900000EBC0033B4C04EB83031B8CD15400EB99
:1066A000C002234603EB8202128C521C00EBC00393
:1066B00004EB83031A8400EBC00304EB83031A8CFE
:1066C000D31702EBD3635B11A2EB431300EBC004BF
:1066D0002C4D05EB840423840A2906D1022200EB09
:1066E000C0032C4604EB83035A8430BD401C0A28A7
:1066F000C2DB002041E000EBC002224B03EB820230
:10670000528CC2BB00EBC00203EB820200EBC00361
:106710001C4C04EB83031B8CD15400EBC0022346BA
:1067200003EB8202128C521C00EBC00304EB8303C8
:106730001A8400EBC00304EB83031A8CD31702EB1B
:10674000D3635B11A2EB431300EBC0040D4D05EBCB
:10675000840423840A2906D1022200EBC0032C46BC
:1067600004EB83035A84012200EBC003054C04EBC5
:1067700083035A84B9E7FFE7401C0A28BBDB00BF4C
:10678000B3E70000702300202DE9F041ADF5107D46
:1067900004460D461646FAF7C7FE002805DA4FF004
:1067A000FF300DF5107DBDE8F0812F48006818B965
:1067B00001202D49086002E04FF0FF30F1E70CB1F5
:1067C00005B126B9002028490860401EE9E702A863
:1067D000FEF7CAFD2548006858B99DF80C000090E6
:1067E0009DF80D30BDF80E2021A1284800F0C8F911
:1067F0000AE09DF80C0000909DF80D30BDF80E20C9
:1068000023A1224800F0BCF93222204905A801F05A
:10681000FAFB074627B1002013490860401EC0E775
:106820009DF8090000909DF80A309DF80B201FA1EB
:10683000224800F0A5F92148F9F732FE8046334698
:1068400042461E4905A801F03AFD33462A46214634
:1068500005A801F034FD05A801F0C4FB00200249A1
:10686000086000BF9DE70000B0010020BC010020CF
:106870002F557372302F4C6F672F25642D25642D93
:1068800025645F72756E2E6C6F6700001C290020F6
:106890002F557372312F4C6F672F25642D25642D72
:1068A00025645F72756E2E6C6F6700002530326450
:1068B0003A253032643A253032640900DC29002060
:1068C000002100EBC002054B03EB8202518400EB78
:1068D000C00203EB82021184704700007023002085
:1068E00092B011AA182126A0FFF74EFF46E000241F
:1068F00035E004EB4410294901EB400040780128C1
:106900002BD104EB441011F81000401C04EB44118F
:10691000224A02F8110004EB4410114611F810004D
:106920003C281ADD402101A8F9F79DFD04EB441035
:106930001A4901EB4000821C19A101A800F020F9BE
:1069400001A8F9F7ADFD054611AA294601A8FFF7F0
:106950001BFF01201949087000BF601CC4B2142C31
:10696000C7DB16480078012802D1FDF76FF801E077
:10697000FDF71CF84FF47A70FDF7C0FEB7E7000092
:106980005461736B5761746368446F673A204A6F50
:10699000696E20696E21210A000000001F2C002072
:1069A0005461736B5761746368446F673A20257351
:1069B00020666C65657421210A000000EC0100204E
:1069C0000146142901DA002902DA4FF0FF3070473E
:1069D00001EB4110064A02EB40004078012805D146
:1069E000002001EB4112024B03F812000020EEE7F9
:1069F0001F2C002010B5FCF7DFFF10BD70B5054659
:106A000015B94FF0FF3070BD002425E004EB4410B1
:106A1000144901EB4000407801281BD0002004EB12
:106A20004411104A02F81100012004EB441102EB5A
:106A3000410148702846F9F733FD064604EB44113E
:106A4000084A02EB4101881C32462946F9F7F2FC5C
:106A50002046D8E7601C44B2142CD7DB4FF0FF303F
:106A6000D1E700001F2C002001468869C0F3C00058
:106A700070470146886900F0100008B9086870473F
:106A80004FF0FF30FBE700BF826902F02002002ACE
:106A9000FAD10160704701468869012222EA10108C
:106AA0007047F0B504460E4615461F46204600F0D6
:106AB0001EF8B6EB051F05D2206B40F020002063C6
:106AC0006D0803E0206B20F020002063F000B0FB95
:106AD000F5F0401C43089809606203F03F00A06293
:106AE000E7620020A061204600F011F8F0BD00BF71
:106AF000816901F008010029FAD1C16A21F0100171
:106B0000C162016B40F20132914301637047C16A77
:106B100041F01001C162016B40F201321143016387
:106B2000704741647047826B0A4382637047024634
:106B300009B1106C7047D06BFCE7816841F001012E
:106B4000816070470121C16070470121C0F8001CBD
:106B5000704701607047816841F0020181607047B1
:106B60000149C0F8001C704751E5CC1A00BF03482A
:106B7000806900F001000028F9D1704700F00A4058
:106B80000FB4084B10B504A902AA039800F0D8F876
:106B9000044602A9002000F06AFC204610BC5DF803
:106BA00014FB00006F7400002DED020B019820F023
:106BB000004001909DED000B02B0704702E008C854
:106BC000121F08C1002AFAD170477047002001E067
:106BD00001C1121F002AFBD1704700002DE9FF5FA1
:106BE000DDE90220010DDDF838B0024318D044F68B
:106BF0001050A1F2FF3141430D140F98012820D00D
:106C0000A5EB0B00401C5FEA000A4FF00004474E62
:106C1000DFF81C91A046504616D5CAF1000728E0BF
:106C20000F98012443A2012808D0002100980F9B4F
:106C3000C0E90021C0E90243BDE8FF9F6FEA0B01F4
:106C4000F4E7CBF10000DEE7074612E0F80707D0D3
:106C50002246334640464946F9F711FD80468946AB
:106C60002246334610461946F9F709FD04460E46FA
:106C70007F10002FEAD1DDE90201BAF1000F424690
:106C80004B4602DAF9F7FBFC01E0F9F76AFD04462E
:106C90000E460022284BF9F7EBFD03D84FF0FF30EA
:106CA000014607E00022254B20463146F9F740FC1B
:106CB000F9F7C6FD102409E0002C0ADB0A220023A4
:106CC000F9F768FB019B30321A55641E50EA010245
:106CD000F2D1641C019AC4F1110314440F9A012AE1
:106CE00003D0012208430DD10AE0084304D000205C
:106CF0004FF0110B0F9080E7A3EB0B056D1E0DE01D
:106D00005B4504DD4FF0000205F1010504E003DA04
:106D10004FF00002A5F10105002AECD000980F9970
:106D2000C0E90231C0E9004586E7000000002440C8
:106D30000000F03F300000000000F0430000E03FA2
:106D40002DE9FF4F95B09B468946064600250FE288
:106D5000252877D100242746F84A0121059400E030
:106D6000044316F8013F203B01FA03F01042F7D12B
:106D700030782A2811D06FF02F033078A0F130023C
:106D8000092A16D8059A44F0020402EB820203EBAA
:106D900042021044761C0590EFE759F8042B059247
:106DA000002A03DA504244F40054059044F00204EF
:106DB000761C30782E2816D116F8010F44F0040402
:106DC0002A280DD06FF02F023078A0F13003092B64
:106DD00009D807EB870302EB4303C718761CF3E7D8
:106DE00059F8047B761C30786C280FD006DC4C28D0
:106DF00017D068280DD06A2814D104E0742810D068
:106E00007A280FD10DE044F400140AE044F4801411
:106E100001E044F440147278824202D104F58014F7
:106E2000761C761C307866280BD013DC582877D077
:106E300009DC002875D04528F6D04628F4D047282C
:106E40001AD19DE118E0632835D0642879D06528EF
:106E500012D195E1702873D008DC6728F1D0692839
:106E60006FD06E280DD06F2806D1B5E073282CD0D6
:106E7000752875D0782874D05A46179990476D1C9C
:106E800075E1C4F30250022809D003280DD0D9F8C7
:106E9000001004280DD00D6009F1040967E1D9F84C
:106EA0000010EA17C1E90052F6E7D9F800100D808A
:106EB000F2E70D70F0E719F8041B8DF800100020C0
:106EC0008DF80100EA46012003E059F804AB4FF0C9
:106ED000FF3061074FF0000102D40DE008F101011D
:106EE0008846B9420FDA8045F8DB1AF80810002905
:106EF000F4D108E008F1010188468142FADB1AF872
:106F000008100029F6D105985B46A0EB080721463A
:106F10003846179A00F094FA284400EB080507E079
:106F20004DE029E10DE01AF8010B5A4617999047F8
:106F3000B8F10108F7D25B4621463846179A13E1AB
:106F400042E00A220092C4F302524FF0000A022AE1
:106F500008D059F804CB032A4FEAEC710AD00DE0AF
:106F600029E02AE009F1070121F00702F2E802C155
:106F7000914609E00FFA8CFC4FEAEC71042A03D128
:106F80004FFA8CFC4FEAEC71002907DA0A4600211F
:106F9000DCF1000C61EB02012D2202E0220504D598
:106FA0002B228DF80420012203E0E20701D02022E9
:106FB000F7E7904659E00A2102E010220DE0102187
:106FC0004FF0000A00910BE010224FF0000A44F04D
:106FD00004040827009203E008224FF0000A009200
:106FE000C4F30252022A05D059F804CB0021032A27
:106FF00008D009E009F1070121F00702F2E802C117
:10700000914605E01FFA8CFC042A01D10CF0FF0C1C
:107010004FF00008220728D5702806D0009B83F087
:10702000100353EA0A0305D00EE040228DF8042035
:10703000012208E05CEA010206D030228DF804202B
:107040008DF8050002229046009B83F0080353EA66
:107050000A030AD15CEA010201D1620705D5302298
:107060008DF804204FF001087F1E582804D034A06A
:1070700003900EA802900DE036A0F9E75346604653
:10708000009AF9F787F984460398825C0298401EBB
:10709000029002705CEA0100F0D1029806A9081A79
:1070A00000F1200A600702D524F4803400E00127B3
:1070B000574502DDA7EB0A0000E0002000EB0A01C3
:1070C000009005984144401A0590E00306D45B46C1
:1070D0002146179A059800F0B3F90544002706E009
:1070E00001A85A46C05D179990476D1C7F1C474503
:1070F000F6DBE0030CD55B462146179A059800F0B5
:107100009FF9054404E030205A46179990476D1CBA
:107110000099481E00900029F5DC08E002980299C9
:107120005A460078491C0291179990476D1CBAF194
:107130000001AAF1010AF1DC65E100000928010063
:1071400030313233343536373839616263646566DD
:10715000000000003031323334353637383941429F
:10716000434445460000000000F058F90544761CF1
:10717000307800287FF4ECAD19B02846BDE8F08FD8
:10718000620700D4062709F1070222F0070CFCE889
:107190000223E14603F000485FEA080C02D00FF238
:1071A000702C0DE05FEA045C02D50FF2682C07E05A
:1071B0005FEAC47C02D00FF2602C01E0AFF2700CE9
:1071C0004FF0FF3823F00043CDF850C065280CD0B5
:1071D00006DC452809D046281DD047283DD13DE092
:1071E000662818D067287ED138E00021112F01DBF6
:1071F000112000E0781CCDE9000106A90EA8FFF7D8
:10720000EDFCDDE90F010E9A03910021009207F1D8
:10721000010A04914DE04FF000400097CDE90110C4
:1072200006A90EA8FFF7DAFCDDE90F0203920E9B18
:1072300011990022DDF80CA00093049211B9791C79
:1072400000EB010AB7EB0A0004D4C0F1FF3007F1EC
:10725000010A0490AAEB0700019044E0012F00DA34
:1072600001270021112F01DD112000E03846CDE972
:10727000000106A90EA8FFF7B1FCDDE90F010E9A87
:107280000391002104910092BA4621070CD403997E
:10729000514500DA8A46BAF1010F05DD009AAAF1DC
:1072A0000101515C302908D0B84202DA10F1040F14
:1072B00006DA0121CDE9011015E0AAF10101E9E7A3
:1072C000002805DC049901440491AAEB000102E0C6
:1072D000411C514500DD8A460499401A401C01902A
:1072E0004FF000400290200704D40198504501DB84
:1072F000CDF8048000208DF84F0002980DF14F0763
:10730000B0F1004F25D02B200E9002984FF00208CC
:1073100000280CDA404202902D200E9007E00A214E
:107320000298F9F7EFF83031029007F8011DB8F133
:107330000001A8F10108F2DC02980028EFD1791EC3
:107340000E980870307800F0200040F0450007F8F3
:10735000020D12A8C01B00F107081498007800B1B4
:10736000012000EB0A01019801EBE071059841440E
:10737000401A401E0590E00306D45B462146179A4A
:10738000059800F05DF805441498007818B15A4645
:10739000179990476D1CE00324D55B462146179A48
:1073A000059800F04DF805441CE00498002807DB20
:1073B000DDE90301884203DD0098405C179901E094
:1073C000179930205A469047049805F10105401C52
:1073D00004900198401E019004D12E205A4617991E
:1073E00090476D1CBAF10001AAF1010ADDDC05E04D
:1073F00017F8010B5A46179990476D1CB8F1000118
:10740000A8F10108F4DC5B462146179A0598ABE623
:107410002D0000002B000000200000002DE9F041AD
:10742000044600251E461746880404D405E0394664
:107430002020B0476D1C641EF9D52846BDE8F081B8
:107440002DE9F041044600251E469046C80301D5AB
:10745000302700E02027880404D505E0414638465F
:10746000B0476D1C641EF9D52846BDE8F0810A6856
:10747000531C0B60107070472DE9F041044688469C
:107480000020E070401E60634146204601F0A2FCEF
:1074900010B10420BDE8F08104F2362001F0ABFA0F
:1074A000074694F83850EB2D03D0E92D01D0E82D94
:1074B00034D14AF65520874208D108221BA104F195
:1074C0008A0001F009FB08B90020E3E704F143005A
:1074D00001F091FA0646701E3040F8B9B6F5007F0B
:1074E0001CDBB6F5007F19DC4520055DB5B1681ED3
:1074F000284098B94820005D012803D04820005D4D
:1075000002280BD104F1490001F075FA30B104F101
:107510004E0001F070FA08B10020BBE74AF6552092
:10752000874201D10220B5E70320B3E74641543337
:107530003220202000000000024600E0521C10789B
:1075400010B110788842F9D110787047F0B5034631
:107550000D461E68986A021D680A7789B0FBF7F429
:1075600000BF02CA09B90020F0BD8C4200D202E07F
:10757000641A121DF5E700BF10682044F4E70246C4
:10758000891ED069801E884201D800207047538927
:10759000106B03FB0100F9E72DE9F04780460C462C
:1075A00004F11A0001F027FA10B10020BDE8F087BD
:1075B000207800F03F00401E00EB800101EBC00589
:1075C0004FF00109002621E01849895D081901F0F2
:1075D00012FA0746B9F1000F11D0FF2D0BD838462B
:1075E00000F0A6FF824629466D1C38F8110000F015
:1075F0009FFF824501D00020D8E7B94605E04FF64D
:10760000FF70874201D00020D0E7761C0D2EDBD31F
:10761000207800F0400038B1B9F1000F04D038F8FC
:10762000150008B10020C1E70120BFE7D096000097
:107630002DE9F04782468846DAF80040B8F1000F9D
:1076400006D1276917B1E069B84215D8012713E0C0
:107650004146504601F0F4F80546022D02D20120C1
:10766000BDE8F087681C08B92846F9E7E069A84238
:1076700001D92846F4E74746606908B90020EFE7DA
:107680000026474518D17E1CE069B04200D802268A
:107690003146504601F0D4F80546012D01D0681C52
:1076A00008B92846DCE73DB12569022D03D3E0691E
:1076B000A84200D92F460026E6B93E4600BF761CF8
:1076C000E069B04204D80226BE4201D90020C7E7D3
:1076D0003146504601F0B4F8054605B909E0012DE0
:1076E00001D0681C08B92846BAE7BE42E7D100209D
:1076F000B6E700BF4FF0FF323146204601F084FB71
:107700008146B9F1000F08D1B8F1000F05D032461B
:107710004146204601F078FB8146B9F1000F0DD1BA
:107720002661E069801E6169814202D86069401E5D
:107730006061207940F00100207107E0B9F1010F8C
:1077400002D14FF0FF3000E001200646304687E7C7
:107750002DE9F34F83B08146049800680090D9F872
:107760000000C768002500BF684601F018FD0290C0
:107770000298401C18B9062005B0BDE8F08F0298A9
:10778000B0F5803F05D30298020C28466D1C27F8FF
:107790001020029884B2202C03DB2F2C01D05C2C0B
:1077A00000D111E0802C06DA214693A0FFF7C4FE39
:1077B00008B10620E0E7FF2D01D30620DCE72846CC
:1077C0006D1C27F81040CFE700BF202C01DA0426FB
:1077D0000CE0002602E00098401C00900098007821
:1077E0002F28F8D0009800785C28F4D000990498ED
:1077F0000160012D04D1681E37F810002E280BD02F
:10780000022D24D1681E37F810002E281FD1A81E83
:1078100037F810002E281AD1002027F815008046CE
:107820000AE0A84501D22E2100E0202109F1200024
:1078300000F8081008F10108B8F10B0FF1D346F079
:10784000200109F1200000F80810002094E708E06A
:10785000681E37F81040202C02D02E2C00D002E0F9
:107860006D1E002DF4D100BF002027F815000DB9C2
:10787000062081E74FF0000A01E00AF1010A37F81B
:107880001A002028F9D0BAF1000F03D137F81A00F6
:107890002E2801D146F0030600E06D1E25B1681EBA
:1078A00037F810002E28F8D10B22202109F12000F2
:1078B00001F031F94FF00008C3460820019000BFE5
:1078C00050460AF1010A37F8104004B968E0202C4C
:1078D00003D02E2C04D1AA4502D046F00306EFE7D0
:1078E0000198804501D2AA4516D101980B2802D1F2
:1078F00046F0030654E0AA4501D046F00306AA4527
:1079000000D94DE0AA464FF008080B2001904FEA3D
:107910008B604FEA106BD3E7802C0EDB46F002063B
:1079200040F2B511204600F0E3FD044604F080006B
:1079300018B104F07F0033490C5CFF2C10DD019876
:10794000401E404504D846F00306DDF80480B7E742
:107950002212404608F1010809F120010A5418E0FA
:1079600024B1214628A0FFF7E7FD18B15F2446F0B7
:1079700003060EE0412C03DB5A2C01DC4BF0020B1A
:10798000612C06DB7A2C04DC4BF0010BA4F1200007
:1079900084B2404608F1010809F120010C548FE738
:1079A00000BF99F82000E52802D1052089F82000C1
:1079B0000198082803D14FEA8B604FEA106B0BF057
:1079C0000C000C2803D00BF00300032801D146F073
:1079D000020606F0020048B90BF0010008B146F0BB
:1079E00010060BF0040008B146F008062B2000F842
:1079F00009600020C0E60000222A3A3C3E3F7C7F1E
:107A000000000000DD9600002B2C3B3D5B5D00007C
:107A1000014609B1002070470020FCE7014609B18A
:107A2000002070470020FCE72DE9F04104460E4697
:107A3000D4F800800021204600F00DFA0546EDB98B
:107A4000002700BF4046A16901F0C4F9054605B111
:107A500013E0E0690078E52802D0E069007820B9F9
:107A6000781C0746B04201D107E0002701212046DB
:107A700000F0EBF80546002DE4D000BF042D00D146
:107A800007252846BDE8F0812DE9F04704468946E0
:107A9000204601F05FFB10B10120BDE8F0874946A8
:107AA0002046FFF76CFD074667634FF40072002124
:107AB00004F1380001F02FF860894FF40041B1EB78
:107AC000402F01D8084601E06089400206464FF089
:107AD000000800E07608B6F5007F05D9304600F0D2
:107AE000E5FCB0F10008F5D0B6F5007F17D93246B5
:107AF0000021404601F00FF8760A002500E03544E9
:107B00006089A84207D97A1960783346414600F067
:107B100053FA0028F3D0404600F0CEFC10E004F108
:107B200038080126002500E035446089A84207D9BD
:107B30007A1960783346414600F03EFA0028F3D0C7
:107B40006089A84201D00120A7E70020A5E72DE920
:107B5000F0470446D4F800A00021204600F07BF94D
:107B6000064616B13046BDE8F0874FF0FF08C14623
:107B70004FF0FF30E06200BF5046A16901F02AF9E2
:107B8000064606B15EE0E06905780DB9042659E0C5
:107B9000E069C07A00F03F07A771E52D04D007F037
:107BA000080038B10F2F05D04FF0FF084FF0FF301D
:107BB000E06240E00F2F22D12B20005D00F040005A
:107BC00098BB05F0400038B1E06990F80D9005F0E1
:107BD000BF05A8462069E06245450CD1E069407BBD
:107BE000484508D1E169DAF80C00FFF7D5FC10B17F
:107BF000A8F1010000E0FF2000F0FF081BE0B8F151
:107C0000000F05D1E06901F04CFA484500D119E0B8
:107C10002B20005D00F0010040B90B2204F120018F
:107C2000E06900F059FF08B90CE004E04FF0FF08EC
:107C30004FF0FF30E0620021204600F006F80646D3
:107C4000002E99D000BF30468DE72DE9F041044663
:107C500088462768206900F12006B6F5001F01D389
:107C60000020A061A06910B90420BDE8F081C6F32E
:107C70000800002845D1A069401CA061606938B99E
:107C80003889B0EB561F3CD80020A0610420ECE7F7
:107C90007889401E00EA562098BB2046616900F0B2
:107CA000CFFD0546012D01D80220DEE7681C08B98A
:107CB0000120DAE7F869A8421DD8B8F1000F03D116
:107CC0000020A0610420D0E720466169FFF7B0FCE6
:107CD00005460DB90720C8E7012D01D10220C4E7F0
:107CE000681C08B90120C0E729463846FFF7CCFEDA
:107CF00008B10120B9E7656129463846FFF73FFC26
:107D0000A0612661C6F3080107F138000844E0616C
:107D10000020AAE72DE9FE4F044626682B20005DCF
:107D200000F0A00010B10620BDE8FE8F4FF0000962
:107D300001E009F10109F06830F819000028F8D1D4
:107D40000C2204F12001684600F0D8FE9DF80B00DB
:107D500000F0010028B340212B2001554FF001080D
:107D60000EE04346694604F12000F26800F002FD8F
:107D70002046FFF7ECFE054605B104E008F10108D6
:107D8000B8F1640FEDD300BFB8F1640F01D1072043
:107D9000CAE7042D01D02846C6E79DF80B102B201A
:107DA00001559DF80B0000F0020030B109F10C0004
:107DB0000D21B0FBF1F0401C00E0012007463946E0
:107DC0002046FFF731FE05464DBB781E071E26D024
:107DD0002069A0EB4711204600F03DF80546F5B9B3
:107DE00004F1200001F05DF9824600BF3046A16930
:107DF00000F0F0FF054605B110E0FAB2E169534624
:107E0000F06801F09DF80120F07000212046FFF796
:107E10001CFF054615B9781E071EE7D100BFC5B97E
:107E20003046A16900F0D6FF054695B92022002111
:107E3000E06900F070FE0B2204F12001E06900F01F
:107E40005DFE2B20005D00F01800E1690873012041
:107E5000F070284668E72DE9F04104460D46266893
:107E6000B5F5001F02D205F01F0010B10220BDE8D9
:107E7000F0812561A7681FB93078032800DBF76A15
:107E800047B93089B0EB551F01D80220EFE7F06AFF
:107E9000A0611CE070894FEA402811E03946204675
:107EA00000F0CEFC0746781C08B90120DFE7022F5E
:107EB00002D3F069B84201D80220D8E7A5EB080543
:107EC0004545EBD239463046FFF759FBA061676163
:107ED000A06908B90220CAE7A06900EB5520A0619B
:107EE000C5F3080106F138000844E0610020BEE750
:107EF00070B5054665B9FDF7C9FA044634B10120ED
:107F0000FDF774FCFF20FDF78EFC01E0002070BD42
:107F100000BF0120FBE72DE9F04106460F4615465C
:107F20002EBB37B1012F1AD0022F0FD0032F1BD138
:107F300011E00020FDF770FCFDF782FC08B9002479
:107F400000E001240120FDF767FC0FE04FF4007012
:107F5000288000240AE008202880002406E0FDF79D
:107F600055FA2860002401E0042400BF00E0012449
:107F70002046BDE8F0812DE9F04106460F469046C7
:107F80001C4614B90420BDE8F0816EB9E2B2414646
:107F90003846FDF75FFB054625B1FF20FDF743FCA2
:107FA0000120F0E70020EEE70420ECE7014609B9E4
:107FB000002070470120FCE72DE9F04105460E4600
:107FC0001746984665B908F0FF0239463046FDF776
:107FD0005DFC044614B90020BDE8F0810120FBE7F8
:107FE0000420F9E738B50546284600F018F904469C
:107FF0003CB96946284601F0F8F804460CB900205F
:108000002860204638BD2DE9F74F90B0044616464B
:108010001CB9092013B0BDE8F08F06F03F063246C8
:1080200003A911A800F080FD0546002D75D1039825
:1080300004904FF4007000F039FA8346BBF1000F52
:1080400001D11120E6E70398C0F80CB004A81199FB
:1080500000F002FB05462DB99DF83B0000F08000C2
:1080600000B1062506F01C00002857D045B1042DAC
:1080700003D104A8FFF74EFE054646F008060AE0C5
:108080009DF8160000F0110008B1072503E006F086
:10809000040000B10825002D51D106F00800002889
:1080A0004DD000F03DFC01900B9901F10E000199BB
:1080B00000F0E5FF0B9901F11600019900F0DFFFD8
:1080C0000B99039800F078FC814620200B99C87228
:1080D00000220B99039800F0C0FF0B9901F11C00DE
:1080E000002100F0CCFF01200399C870B9F1000F06
:1080F00025D00398D0F834A00022494604A800F007
:108100005FFF0546DDB95146039800F063FE054662
:10811000A9F101000399086111E07BE07DB99DF8A8
:10812000160000F0100008B1042508E006F0020077
:1081300028B19DF8160000F0010000B107254DB9E7
:1081400006F0080008B146F040060398406B206234
:108150000B986062002D5AD10B99039800F02CFC0B
:10816000A0600B9901F11C0000F039FCE0600020D8
:10817000A062039820600398C088A0802674002025
:108180006074E06160614FF40072002104F12C0022
:1081900000F0C1FC06F0200058B3E06848B3E06886
:1081A00060610398408940020290A768D4F80C806F
:1081B0000DE03946204600F043FB0746012F00D86A
:1081C0000225781C00B901250298A8EB000815B912
:1081D00002988045EDD8A7615DB9C8F3080040B1A9
:1081E00039460398FFF7CBF98246BAF1000F01D167
:1081F00002250CE00AEB5820E061E2690399487817
:10820000012304F12C01FFF7B6FE00B10125584609
:1082100000F052F90DB1002020602846FAE6F8B5CA
:1082200004466946204600F0E0FF0646002E44D191
:10823000207C00F0400000283FD0207C00F080002F
:1082400070B1E26900994878012304F12C01FFF72D
:10825000B3FE08B10120F8BD207C00F07F0020743F
:1082600000F05EFB0746216A009800F0B3FD064669
:108270001EBB656AE87A40F02000E8722946A268D1
:10828000206800F0EAFE05F11C00E16800F0F7FE4E
:10829000394605F1160000F0F2FE002105F112004A
:1082A00000F0F9FE01200099C870009800F00AFF64
:1082B0000646207C00F0BF0020743046CBE72DE955
:1082C000FF4F83B0044615469B460498009000205B
:1082D000CBF8000001A9204600F087FF0290029829
:1082E00010B9607C029018B1029807B0BDE8F08F19
:1082F000207C00F0020008B90720F6E700BF6069A3
:1083000028446169884202D26069C0F1FF35C3E048
:10831000A08AC0F3080000287DD101984089401E42
:10832000616900EA512ABAF1000F26D1606938B9B3
:10833000A76897B900212046FFF77AF907460CE0B5
:10834000A06A28B120466169FFF700F9074604E0FA
:108350002046A169FFF76CF9074607B99FE0012F96
:1083600002D102206074C0E7781C10B9012060744B
:10837000BBE7A761A06800B9A760207C00F080007F
:1083800078B1E26901994878012304F12C01FFF7E3
:1083900013FE10B101206074A7E7207C00F07F007D
:1083A0002074A1690198FFF7EAF8064616B9022081
:1083B00060749AE756444FEA5529B9F1000F2BD063
:1083C0000AEB090001994989884203D9019840893B
:1083D000A0EB0A09019948784B4632460099FFF70D
:1083E000EBFD10B1012060747FE7E069801B484518
:1083F0000ED2E069801B009A02EB40214FF400721C
:1084000004F12C0000F07AFB207C00F07F00207447
:108410004FEA49282BE013E0E069B0420FD0E16851
:10842000606988420BD2019948780123324604F1F1
:108430002C01FFF7A0FD10B10120607455E7E66143
:10844000A08AC0F30800C0F50078A84500D9A84666
:10845000A18AC1F3080204F12C0150184246009988
:1084600000F04CFB207C40F08000207400BFA5EBA6
:108470000805DBF800004044CBF8000000984044B9
:108480000090606940446061E1686069884201D998
:10849000606900E0E068E060002D7FF439AF00BF64
:1084A000207C40F04000207400201EE710B50446F8
:1084B000204600F0DBFA10BD10B50446204600F05F
:1084C00031F910BD10B502460020084B802A01DAB0
:1084D000104609E040F2B514A14205D1FF2A03DCA1
:1084E000A2F1800433F8140010BD00008C97000046
:1084F00010B5024600200D4B802A01D290B213E045
:10850000B2F5803F10D240F2B514A1420CD1002048
:1085100001E0441CA0B2802803DA33F810409442F2
:10852000F7D100F18004E0B210BD00008C9700008C
:1085300070B5B0F5803F4DD281B2B1F5805F01DA00
:10854000254E00E0254E324600BF32F8023B0BB10B
:10855000994200DA3CE032F8024B2512E4B21E19CF
:108560008E4230DD092D2CD2DFE805F005090F130E
:10857000171B1F232700CE1A32F8161021E0CE1A3F
:1085800006F001068E1BB1B21BE0A1F11006B1B2DC
:1085900017E0A1F12006B1B213E0A1F13006B1B2AB
:1085A0000FE0A1F11A06B1B20BE001F10806B1B279
:1085B00007E0A1F15006B1B203E0A1F5E356B1B274
:1085C00000BF00BF04E0002DBFD102EB4402BCE7B6
:1085D00000BF084670BD00008C9800007E9A000025
:1085E0002DE9FF4107460D4600213846FEF744FFBE
:1085F0000646022E06D0032E00D21DB9304604B026
:10860000BDE8F08100BF00240AE007F5FB7101EB33
:10861000041101F1080000F0E2F94DF82400641C97
:10862000042CF2D30DB1681E00E00020044600BF08
:108630005DF8240028B15DF824103846FEF71CFFD1
:1086400000E0032006462DB9022E03D3601C044629
:108650000428EDD33046D2E72DE9F34104462768DC
:10866000019800782F2806D0019800785C2802D065
:10867000B869A0600DE002E00198401C01900198EB
:1086800000782F28F8D0019800785C28F4D00020DA
:10869000A06001980078202808D280212B20015565
:1086A00000212046FFF7D7FB054637E000BF01A9B0
:1086B0002046FFF74DF8054605B12EE02046FFF7AE
:1086C00046FA05462B20065D95B1042D0FD106F024
:1086D000200040B106F0040000B9E8E780212B201B
:1086E0000155002503E006F0040000B9052514E05B
:1086F00006F0040000B110E0A07900F0100008B905
:1087000005250AE0208AC0F3080207F13800111895
:10871000384600F051F9A060C9E700BF2846BDE81F
:10872000FC81000010B5002821D0114B0022001F51
:10873000196803E0814203D80A4649680029F9D143
:1087400052B11368841A9C4204D100681844106026
:10875000104602E0506000E0186039B102680B1A60
:10876000934203D10B681A4402604968416010BD0E
:10877000F00100202DE9FF4F83B0804691461E4650
:108780000B224046049900F0B9F9052E18D9374656
:1087900011E039F802BB00250BE0584667F35F0093
:1087A00007464FEA6B0B07F4803008B12348474077
:1087B0006D1C102DF1D3B9F800000028E9D13E4618
:1087C000072500BF06F00F0000F1300ABAF1390F9B
:1087D00003DD0AF1070000F0FF0A28466D1E01A91B
:1087E00001F800A03609002EECD17E204855002467
:1087F0000AE018F80400FFF70BF920B1681EA04248
:1088000000D107E0641C641CAC4203D218F80400D9
:108810002028EED100BF00BF082D04D228466D1CD1
:1088200001A9085C00E020202146641C08F8010032
:10883000082CF1D307B0BDE8F08F00002110010033
:108840002DE9F04781460C46D9F80050022C02D39E
:10885000E869A04202D84FF001085EE04FF0FF380F
:108860002878012804D002282CD0032851D13CE0DC
:10887000264606EB5606A86A00EB5621284600F06D
:10888000A9FA00B148E03046761CC0F3080105F1B2
:108890003800475CA86A00EB5621284600F09AFA97
:1088A00000B139E0C6F3080105F13800405C47EA41
:1088B000002704F0010008B1380901E0C7F30B00FC
:1088C000804629E0A86A00EB1421284600F082FACD
:1088D00000B121E040F2FF1101EA440205F1380144
:1088E000501800F088F8804616E0A86A00EBD41112
:1088F000284600F06FFA00B10EE040F2FF1101EAE5
:10890000840205F13801501800F069F820F0704831
:1089100002E04FF0010800BF00BF4046BDE8F0870D
:108920000EB56846FCF720FDC0B9BDF80600A0F200
:10893000BC7040069DF8051040EA41509DF80410B7
:1089400040EA01409DF8031040EAC1209DF8021062
:1089500040EA41109DF8011008430EBD0048FCE7B5
:108960002252A55670B504464FF0FF3026683146B6
:10897000324601B970BD00BF12F8013B202B01D374
:108980003A2BF9D13A2B11D101250E78302E08DB84
:108990000E78392E05DC8E1C964202D10E78A6F197
:1089A0003005012D01DA28462260E3E7014E3078D8
:1089B00000BFDFE78A01002070B505460C4604F1D0
:1089C0001A0000F018F806462878032805D104F1AB
:1089D000140000F010F846EA0046304670BD01462B
:1089E000C8788A7842EA00204A7842EA00200A7869
:1089F00042EA00207047014648780A7842EA00209F
:108A00007047000088B006A90FA0F8F70DFDF7F732
:108A100039FCFBF75BF9032000214FF400720E4B89
:108A2000CDE90132CDE90310022003460B4A009044
:108A30000B48FBF755FB07AA0AA10220FBF76CFCC9
:108A4000FBF7FEFA00BFFEE7544D344331323934B0
:108A50004B4350445400000048310020443900206A
:108A6000A10B00005374617274000000F0B50B306C
:108A7000154D20F007010024144A0FE003688B42D3
:108A80000BD38B4205D95E1A43184768C3E90067C8
:108A900000E04368136002C004E0021D1068002873
:108AA000ECD12046002802D1286808B10020F0BD92
:108AB000064A07481060074A121A22F00702C0E966
:108AC000002401202860D7E7F4010020F0010020F5
:108AD0004C49002048790020F0B503461D460C465D
:108AE000002000BF15F8017B14F801CBA7EB0C00A8
:108AF000561E321E01D00028F4D0F0BD30B503461A
:108B00000C463AB100BF14F8015B03F8015B551E37
:108B10002A1EF8D130BD10B5034600BF03F8011B73
:108B2000541E221EFAD110BD2DE9F74F84B000214A
:108B3000059801600498FFF715FF0390039800283B
:108B400003DA0B2007B0BDE8F08F9D49039851F878
:108B500020400CB90C20F5E705980460069800F059
:108B6000FE000690207878B16078FFF71FFA07467C
:108B700007F0010040B9069820B107F0040008B1E1
:108B80000A20DFE70020DDE70020207003986070F6
:108B90006078FFF7ADF9074607F0010008B1032040
:108BA000D0E7069820B107F0040008B10A20C9E711
:108BB00000212046FFF714FD0546042D01D10120B8
:108BC000C0E7022D01D30D20BCE7D4F8349004F1A6
:108BD0004300FFF710FFB0F5007F01D00D20B1E793
:108BE00004F14E00FFF707FF064626B904F15C00CA
:108BF000FFF7F5FE064626624820005DA070A078CB
:108C0000012804D0A078022801D00D209AE7A0788E
:108C100046434520005D6081608918B16089411E2E
:108C2000084008B10D208DE704F14900FFF7E3FE8D
:108C30002081207A00F00F0008B10D2082E704F1B6
:108C40004B00FFF7D8FE8246BAF1000F04D104F1C1
:108C50005800FFF7C4FE824604F14600FFF7CBFE42
:108C60008346BBF1000F01D10D206BE70BEB060033
:108C7000218900EB111002900298824501D20D204B
:108C800060E70298AAEB00006189B0FBF1F8B8F147
:108C9000000F01D10D2055E700254A48804500D836
:108CA00003254FF6F570804500D8022540F6F57093
:108CB000804500D801250DB90D2043E708F10200D9
:108CC000E061C4F8249009EB0B00A06202984844CC
:108CD0002063032D13D104F16200FFF78CFE08B16D
:108CE0000D202FE7208908B10D202BE704F1640047
:108CF000FFF775FEE062E0698000019014E02089D2
:108D000008B90D201EE7A06A3044E062022D02D1AE
:108D1000E069400007E0207F00F00100E16901EB1D
:108D2000410100EB51000190216A019800F2FF100F
:108D3000B1EB502F01D20D2004E74FF0FF306061FE
:108D4000206180202071032D2DD104F16800FFF7F0
:108D500052FE012827D109F10101204600F03AF81E
:108D600008BB0020207104F23620FFF744FE4AF6CB
:108D70005521884217D104F13800FFF730FE12491F
:108D8000884210D104F50770FFF729FE0F49884289
:108D900009D104F50870FFF722FE606104F509703F
:108DA000FFF71DFE2061257009480088401C80B235
:108DB00007490880E0800020A06100BFC2E60000F3
:108DC00084010020F5FFFF0F525261417272416130
:108DD0008801002070B504460D460026606BA8424D
:108DE00010D0204600F0B6F906465EB9607801233F
:108DF0002A4604F13801FFF7BEF810B14FF0FF35F5
:108E000001266563304670BD2DE9F04704460D46E6
:108E100016464FF00209022D74D3E069A84271D9B9
:108E20002078012804D0022849D003280DD15EE023
:108E30002F4607EB5707A06A00EB57212046FFF7A4
:108E4000C9FF8146B9F1000F00D075E038467F1C9C
:108E5000C0F3080104F1380001EB000805F001003F
:108E600028B1F1B298F8000061F31F1000E030461D
:108E700088F800000120E070A06A00EB572120462E
:108E8000FFF7A8FF8146B9F1000F00D054E0C7F307
:108E9000080104F1380001EB000805F0010010B1F1
:108EA000C6F3071006E098F8000000F0F000C6F3E3
:108EB0000321084388F800000120E0703CE0A06A2C
:108EC00000EB15212046FFF785FF8146B9F1000F21
:108ED00000D031E0B1B240F2FF1202EA450304F1E2
:108EE0003802981800F0D7F80120E07024E0A06A5A
:108EF00000EBD5112046FFF76DFF8146B9F1000F59
:108F000001D019E019E040F2FF1101EA850204F1F5
:108F100038015018FFF763FD66F31B00064640F268
:108F2000FF1101EA850204F138015018314600F0C2
:108F3000A6F80120E07000BF00BF4846BDE8F087FA
:108F40002DE9F04707460C461546984684F80D80F3
:108F50000F20E07200202073002104F11A0000F0BD
:108F60009AF8681E00EB800101EBC009002006465C
:108F7000824600BF4FF6FF70864204D0484609F192
:108F8000010937F810600D4911F80A100819314627
:108F900000F081F80EB94FF6FF760AF10100824623
:108FA0000D28E7D34FF6FF70864202D037F819003C
:108FB00008B945F040052570BDE8F087D09600005F
:108FC0002DE9F04781460E4617464FF00008D9F8C4
:108FD0000040022E02D3E069B04202D80220BDE870
:108FE000F08767B100BF4FF0FF3239462046FFF7E8
:108FF0000BFF8046B8F1000F01D04046EFE700BFFD
:1090000031464846FFF71CFC054605B922E0012D14
:1090100001D10220E3E7681C08B90120DFE7002244
:1090200031462046FFF7F0FE8046B8F1000F01D030
:109030004046D4E7E069801E6169814206D26069DA
:10904000401C6061207940F0010020712E46E069EB
:10905000B042D5D800BF0020C1E770B506460C4627
:109060001546A9B204F11A0000F015F8307803286B
:1090700004D1290C04F1140000F00DF870BD00F8C3
:10908000011B090A00F8011B090A00F8011B090A63
:1090900000F8011B704700F8011B091200F8011BC2
:1090A000704730B5014600200B2200BF431003EB90
:1090B000C01411F8015B6319D8B2531E1A1EF5D102
:1090C00030BD000070B50446204600F043F8054668
:1090D000002D38D1207803282ED1207901282BD1DA
:1090E0004202002104F13800FFF715FD4AF6552130
:1090F00004F23620FFF7CFFF144904F13800FFF7E0
:10910000BEFF134904F50770FFF7B9FF04F50870B7
:109110006169FFF7B4FF04F509702169FFF7AFFF3C
:10912000606A401C60636078012304F13801626B5F
:10913000FEF742FF00202071607800221146FEF702
:10914000EAFE00B10125284670BD0000525261417F
:109150007272416170B504460025E078E8B160782C
:10916000012304F13801626BFEF726FFA0B900204D
:10917000E070A16A606B401A216A88420DD2A07823
:1091800002280AD1236A616BCA186078012304F1AE
:109190003801FEF711FF00E00125284670BD2DE9DA
:1091A000F0410646356815F8014B2046FEF730FCC5
:1091B00060B115F8017B3846FEF730FC18B94FF066
:1091C000FF30BDE8F08107EB042084B24CB140F2DF
:1091D000B5112046FFF776F9044614B94FF0FF3079
:1091E000EFE7A04635604046EBE770B504460D4614
:1091F00009268CB1206878B12068007860B1A08819
:109200002168C988884207D121684878FEF7CEFED8
:1092100000F0010000B900260EB9206800E000202F
:109220002860304670BD0000004000401000000083
:1092300000800540100000000050004011000000B8
:109240000090054011000000006000401200000086
:1092500000A0054012000000007000401300000054
:1092600000B0054013000000004002401400000060
:1092700000C0054014000000005002402E00000015
:1092800000D005402E000000006002402F000000CA
:1092900000E005402F000000007002403000000098
:1092A00000F005403000000000D003404600000000
:1092B0000000064046000000001006404700000085
:1092C0000020064048000000003006407F000000FB
:1092D000004006408000000000500640840000006E
:1092E000006006408C0000000040004010000000BC
:1092F00000800540100000000050004011000000F8
:1093000000900540110000000060004012000000C5
:1093100000A0054012000000007000401300000093
:1093200000B005401300000000400240140000009F
:1093300000C0054014000000005002402E00000054
:1093400000D005402E000000006002402F00000009
:1093500000E005402F0000000070024030000000D7
:1093600000F005403000000000D003404300000042
:1093700000000640430000000010064044000000CA
:109380000020064045000000003006405800000064
:109390000040064059000000005006405C000000FC
:1093A0000060064064000000007006406C00000091
:1093B000008006406D000000009006407F00000025
:1093C00000400040008005400050004000900540F3
:1093D0000060004000A005400070004000B0054063
:1093E0000040024000C005400050024000D005404F
:1093F0000060024000E005400070024000F00540BF
:1094000000D0034000000640001006400010064057
:109410000020064000200640003006400030064094
:109420000040064000400640005006400050064004
:109430000060064000600640007006400070064074
:1094400000800640008006400090064000900640E4
:1094500000070000000600000005000000040000F6
:1094600000030000000200000001000000000000F6
:109470000000000018ED00E01CED00E020ED00E031
:1094800000E400E004E400E008E400E00CE400E0B4
:1094900010E400E014E400E018E400E01CE400E064
:1094A00020E400E024E400E028E400E02CE400E014
:1094B00030E400E034E400E038E400E03CE400E0C4
:1094C00040E400E044E400E048E400E04CE400E074
:1094D00050E400E054E400E058E400E05CE400E024
:1094E00060E400E064E400E068E400E06CE400E0D4
:1094F00070E400E074E400E078E400E07CE400E084
:1095000080E400E084E400E088E400E000E100E0C2
:1095100004E100E008E100E00CE100E010E100E01F
:1095200080E100E084E100E088E100E08CE100E01F
:1095300090E100E000E200E004E200E008E200E088
:109540000CE200E010E200E080E200E084E200E0F3
:1095500088E200E08CE200E090E200E00000010020
:1095600002000100030001000200010004000100EC
:1095700002000100030001000200010005000100DB
:1095800002000100030001000200010004000100CC
:1095900002000100030001000200010006000100BA
:1095A00002000100030001000200010004000100AC
:1095B000020001000300010002000100050001009B
:1095C000020001000300010002000100040001008C
:1095D0000200010003000100020001000700010079
:1095E000020001000300010002000100040001006C
:1095F000020001000300010002000100050001005B
:10960000020001000300010002000100040001004B
:109610000200010003000100020001000600010039
:10962000020001000300010002000100040001002B
:10963000020001000300010002000100050001001A
:10964000020001000300010002000100040001000B
:1096500002000100030001000200010001000000FF
:109660007856341201003F0001001800E80501009F
:1096700001001000140002000A0001003F00010078
:10968000010005000100180078000100040001003D
:10969000040018000800010004000100010001009E
:1096A000800001001600010001008000010001009F
:1096B000010040005800E80301001A720100100088
:1096C00001000800E80328008002080040000A1991
:1096D00001030507090E10121416181C1E809A4566
:1096E000418E418F804545454949498E8F909292E0
:1096F0004F994F555559999A9B9C9D9E9F41494F13
:1097000055A5A5A6A7A8A9AAABACADAEAFB0B1B2FE
:10971000B3B4B5B6B7B8B9BABBBCBDBEBFC0C1C2A1
:10972000C3C4C5C6C7C8C9CACBCCCDCECFD0D1D291
:10973000D3D4D5D6D7D8D9DADBDCDDDEDFE0E1E281
:10974000E3E4E5E6E7E8E9EAEBECEDEEEFF0F1F271
:10975000F3F4F5F6F7F8F9FAFBFCFDFEFF00010063
:10976000040010004000000100020000010002009F
:1097700004000800100020000000000007000000A6
:10978000000000000000000000000000C700FC0016
:10979000E900E200E400E000E500E700EA00EB0099
:1097A000E800EF00EE00EC00C400C500C900E600D0
:1097B000C600F400F600F200FB00F900FF00D6003E
:1097C000DC00A200A300A500A7209201E100ED00AB
:1097D000F300FA00F100D100AA00BA00BF00102384
:1097E000AC00BD00BC00A100AB00BB0091259225E0
:1097F00093250225242561256225562555256325B7
:10980000512557255D255C255B251025142534251C
:109810002C251C2500253C255E255F255A25542531
:1098200069256625602550256C25672568256425F2
:10983000652559255825522553256B256A25182558
:109840000C25882584258C2590258025B103DF00F3
:109850009303C003A303C303B500C403A603980383
:10986000A903B4031E22C603B50329226122B10055
:109870006522642220232123F7004822B000192208
:10988000B7001A227F20B200A025A00061001A03B1
:10989000E0001703F8000703FF0001007801000152
:1098A000300132010601390110014A012E0179010E
:1098B000060180014D004302810182018201840181
:1098C000840186018701870189018A018B018B014F
:1098D0008D018E018F0190019101910193019401FD
:1098E000F60196019701980198013D029B019C01A8
:1098F0009D0120029F01A001A001A201A201A401DB
:10990000A401A601A701A701A901AA01AB01AC010D
:10991000AC01AE01AF01AF01B101B201B301B301BE
:10992000B501B501B701B801B801BA01BB01BC016D
:10993000BC01BE01F701C001C101C201C301C401E4
:10994000C501C401C701C801C701CA01CB01CA01D1
:10995000CD011001DD0101008E01DE011201F301D4
:109960000300F101F401F401F801280122021201BF
:109970003A020900652C3B023B023D02662C3F0285
:1099800040024102410246020A01530240008101A5
:109990008601550289018A0158028F015A029001FD
:1099A0005C025D025E025F02930161026202940149
:1099B0006402650266026702970196016A02622CE0
:1099C0006C026D026E029C01700271029D017302B5
:1099D00074029F0176027702780279027A027B0292
:1099E0007C02642C7E027F02A60181028202A90110
:1099F0008402850286028702AE014402B101B201EF
:109A000045028D028E028F0290029102B7017B0304
:109A10000300FD03FE03FF03AC0304008603880379
:109A200089038A03B1031103C2030200A303A30342
:109A3000C4030803CC0303008C038E038F03D803F5
:109A40001801F2030A00F903F303F403F503F60324
:109A5000F703F703F903FA03FA0330042003500471
:109A60001007600422018A043601C1040E01CF04EC
:109A70000100C004D00444016105260400007D1DDE
:109A80000100632C001E9601A01E5A01001F08064B
:109A9000101F0606201F0806301F0806401F060676
:109AA000511F0700591F521F5B1F541F5D1F561F78
:109AB0005F1F601F0806701F0E00BA1FBB1FC81F64
:109AC000C91FCA1FCB1FDA1FDB1FF81FF91FEA1FB0
:109AD000EB1FFA1FFB1F801F0806901F0806A01F20
:109AE0000806B01F0400B81FB91FB21FBC1FCC1F4F
:109AF0000100C31FD01F0206E01F0206E51F010080
:109B0000EC1FF31F0100FC1F4E21010032217021C8
:109B10001002842101008321D0241A05302C2F0447
:109B2000602C0201672C0601752C0201802C640157
:109B3000002D260841FF1A03000000004141424267
:109B40002C25302E32662C25302E32662C25302ED8
:109B500032662C25302E32662C25302E32662C258E
:109B6000302E32662C25302E32662C25302E326671
:109B70002C25302E32662C25302E32662C25642C76
:109B800025642C25642C25640A000000AC9B000091
:109B900000000020F8010000A2090000EC9B00007A
:109BA000F801002050970000CC6B000001841A01DE
:109BB000015A0401092C3901170A2D021809164807
:109BC000095E1811D2141008537461727455701024
:109BD0000C45786550617468436F6E665AFF01C129
:0C9BE000E910A914E91C09167B00000024
:0400000500000201F4
:00000001FF
